:020000040000FA
:040000000AEF15F0FE
:0800080049EF15F0186E7F0BA3
:1000100018BC8008F76A240FF66E0800F55018BE69
:1000200000081200000306090C101316191C1F22E9
:1000300025282B2E313336393C3F414447494C4E1D
:10004000515355585A5C5E60626466686A6B6D6FA6
:1000500070717374757678797A7A7B7C7D7D7E7E1B
:100060007E7F7F7F7F002C6A2D6A01D0206E215019
:10007000205ED8A021062D502C5ED8A02D06D89049
:1000800021322032D8902D322C32031C1C6E041CDD
:100090001D6E1C2AD8B41D2A830E276E286A296A71
:1000A0002A6A2B6A266A0F0EEA6E02C0E9FF091C53
:1000B000D5EC02F000D000D0040020502826D8B0A3
:1000C000292A215029262C502A26D8B02B2A2D50F7
:1000D0002B2629509BDF800F196E2B5097DF800F46
:1000E00019261930262602C0E9FFEF500910D8A0C2
:1000F0000918EF6E2704D8B4830E276ED8B41C2AD3
:10010000D8B41D3ED7D71200086A800E346E89EF2E
:1001100000F0206A216A226A236A0A9AF2EC01F04E
:10012000D30FD8B40A8A2D0FC60FF8E20A0FF6E3F0
:100130001C6E1B6A1A6A196A0A0E186EB3EC02F07A
:100140001C501824206E1950216E000ED8B0010EDC
:1001500021261A50226E000ED8B0010E22261B5006
:10016000236E000ED8B0010E2326080606E0F2EC3E
:1001700001F0C60F02E20A0FDBE20AAA0BD0201E32
:10018000211E221E231E202AD8B4212AD8B4222AB6
:10019000D8B4232A20501200086A206E216A0096E3
:1001A0000850D8B40086050E076E270E1D6E100E7F
:1001B0000CD8030E1D6EE80E08D81D6A640E05D813
:1001C0001D6A0A0E02D8205008D01C6E2150196EEC
:1001D0002050186E9CEC02F01850186E074E0096D6
:1001E000085003E0075CD8B008D01850D8A4009697
:1001F00000B603D0300FE5EF01F01200366E2DAEE1
:1002000003D02D0EE5EC01F0106A116A126A136A30
:100210002D8E6A0E2C26D8902D322E322F3213328C
:100220001232113210322C3EF6D72F502C5C2F2672
:100230002C5E2E502D5C2E262D5E086A3AD82E0E8E
:10024000E5EC01F0376AD89010342F6E11342E6E21
:1002500012342D6E13342C6E3736D8902F362E363E
:100260002D362C36373610502F261150D8B0113C71
:100270002E261250D8B0123C2D261350D8B0133C65
:100280002C26D8B0373ED8902F362E362D362C3629
:1002900037363750300FE5EC01F02FC010F02EC08C
:1002A00011F02DC012F02CC013F0362ECBD7D89001
:1002B00012000096085003E100860A0E086E2FC057
:1002C0001BF02EC01AF02DC019F02CC018F0076AD0
:1002D000236A226A216A0A0E206E3FEC02F0072A86
:1002E0000750085CD8A4F4D72050D8A4009600A6E4
:1002F00002D0082C04D02050300FE5EC01F0082E7D
:10030000DED71200206E0750D8B4120020C0E9FFDB
:1003100021C0EAFFEF50D8B41200E5EC01F0204A0A
:10032000212A0706F0D7246E0F0EEA6EE26E025005
:10033000E96E120FE16E800E0A16080E256ED89037
:10034000D8B00A3E12D82432252EFAD7000029BA96
:100350000A300BD800D000D000D0D88006D8065084
:100360001D6E055025EC02F0120029AE0BD0EF50A7
:10037000091029AC0918EF6EE7500910D8A0091828
:10038000E76E0AD0EF500910D8A0091829BC091847
:10039000EF6E091CE71600D029501F0B000F196ED5
:1003A0002850110FD8B0192A000032EF02F0A66AC7
:1003B000A68E0900F55002E002D8FBD71200040017
:1003C0009EA8FDD7AD6ED880120001BA93EF01F060
:1003D00001B4DFEF01F001A205D001B003D001B2FA
:1003E000EE6E120034BEEE501200AA6AA96EA66A22
:1003F000A680A850A94AAA2A1200AA6AA86EA66ACC
:10040000A684550EA76EAA0EA76EA6820400A6B2F9
:10041000FDD7A694A94AAA2A1200E836E8363C0B72
:100420000109C212C009C216C050F80B0209C06E01
:10043000320E31EC02F0C2820400C2B2FDD7C4CF4A
:100440002DF0C3502C6E12001D6A1C6EFF0E1C2670
:100450001D2200D0D8A01200030E196EE70E02D89C
:10046000F5D7196AFD0F186EFF0E00D001D01826BF
:10047000040000D0D8A01926D8A01200F8D71B502D
:100480002318800BF46E1BAE06D0D880000E1856D1
:1004900019561A561B5623AE06D0D880000E205689
:1004A0002156225623561C6A1D6A1E6A1F6A306A2C
:1004B000316A326A336A235022102110201023E05F
:1004C000200EF36ED890183619361A361B36303691
:1004D0003136323633362050305C2150315822507C
:1004E00032582350335809E32050305E2150315A9E
:1004F0002250325A2350335AD8801C361D361E36AD
:100500001F36F32EDFD7F4AE06D0D880000E1C566F
:100510001D561E561F561CC018F01DC019F01EC0D7
:100520001AF01FC01BF030C020F031C021F032C0E3
:1005300022F033C023F01200216A206A100EF36EFD
:100540001934203621361C50205C1D50215805E3FB
:100550001C50205E1D50215AD88018361936F32EB3
:10056000EFD718501200200E246E306A316A326ABA
:10057000336AD89018A00ED0205030262150D8B021
:10058000213C31262250D8B0223C32262350D8B00C
:10059000233C332633323232313230321B321A327C
:1005A00019321832242EE5D71200E988E92AEC1610
:1005B0001200A66AA68E0900F55002E0EE6EFBD787
:1005C0001200F34E02D0E652FCD7E6CFEEFFE82E43
:1005D000FCD71200E466FED7F36EE552F32EFDD78A
:1005E000E6CFEEFFE82EFCD71200610EE75C05E6D1
:1005F0007B0EE75C02E7DF0EE716E650EE6EF5E1F4
:100600001200A66AA68EEE500900F55C02E1F566BE
:10061000FAD71200155011183A6E3ABE30D015BEF6
:1006200017D01450105CD8A0000CD8A4010C1550A1
:10063000115CD8A0000CD8A4010C1650125CD8A0F4
:10064000000CD8A4010C1750135CD8A0000C010CAE
:100650001050145CD8A0000CD8A4010C1150155CEB
:10066000D8A0000CD8A4010C1250165CD8A0000C25
:10067000D8A4010C1350175CD8A0000C010C11AECB
:10068000010C000C155011183A6E3ABE34D015BE4C
:1006900019D01450105CD8A0000CD8A4010C15502F
:1006A000115CD8A0000CD8A4010C1650125CD8A084
:1006B000000CD8A4010C1750135CD8A0000CD8A4CF
:1006C000010C000C1050145CD8A0000CD8A4010C34
:1006D0001150155CD8A0000CD8A4010C1250165C67
:1006E000D8A0000CD8A4010C1350175CD8A0000CA3
:1006F000D8A4010C000C11AE010C000C1450105CBD
:10070000376E19E2376C10C039F014C010F039C0E0
:1007100014F011C039F015C011F039C015F012C035
:1007200039F016C012F039C016F013C039F017C0F6
:1007300013F039C017F01A0E376078D0145276E0F3
:10074000366A1150396E15183B6E118E158E080ED3
:10075000375E08E317C036F016C017F015C016F064
:10076000156AF5D7372607E0D890153216321732BA
:100770003632372EF9D73BAE35D01750135E1650B0
:10078000125A1550115A07E2D880000E135612560D
:100790001156800E391A366C04E01306000E125AF8
:1007A000115A040E376E11660DD012C011F013C02D
:1007B00012F036C013F0366A080E105E2DE3372EA5
:1007C000F2D72AD011BE08D0D8903636133612365A
:1007D0001136102EF7D720D038AC26D036AE24D024
:1007E000366A11D0175013261650122215501122B6
:1007F00006E31132123213323632104A0FD038ACBF
:1008000013D036AE11D0133E0FD0123E0DD0113E94
:100810000BD0D8801390EDD7106A02D038821068C0
:10082000136A126A800E116E39AE119E13501200B7
:100830001150326E15183B6E145053E0105254E0B4
:10084000105E7F0E03E2102603E24DD010264EE22A
:1008500013C030F012C031F0328E158E180E396E82
:10086000136A126A116A0BD01750305C1650315857
:1008700011E3316E326A1750305E0BD004E215502E
:10088000325CF2E007E31750305E1650315A1550D3
:10089000325AD88013361236113630363136323667
:1008A000392EECD711BE07D010521DE03B32100696
:1008B000392A3B36E3D738AC1FD007E21750305EF9
:1008C0001650315A1550325A17E3133E15D0123EC6
:1008D00013D0113E11D0113212321332103E0CD00F
:1008E00005D0388604D03884106A02D03882106867
:1008F000136A126A800E116E3BAE119E13501200E5
:100900001150326E15183B6E1050D8A414503CE0B4
:1009100010267E0E03E3105E03E338D0105E33E34F
:1009200013C030F012C031F0328E158E136A126A85
:10093000116A180E396E32323132303206E31750F6
:100940001326165012221550112211321232133270
:10095000392EF1D711BE07D0133612361136105288
:1009600012E01006323438AC17D016E3133E14D020
:10097000123E12D0113E10D0D880113212321332F2
:10098000103E0AD003D03884106A02D03882106832
:10099000136A126A800E116E3BAE119E1350120044
:1009A000126A136A10C036F013C010F036C013F08C
:1009B00012C036F011C012F036C011F0960E396E2A
:1009C0003B6A10AE07D0D880000E1356125611564F
:1009D00010563B8E105218E038AC0DD013AE0BD031
:1009E000123E09D0113E07D0103E05D0D8801032FB
:1009F00011321232392A080E392612C013F011C0F2
:100A000012F010C011F015D0116613D0080E395E27
:100A1000125005E1080E395E135011E0136A116E91
:100A200013C012F0136A05D0D8901336123611365F
:100A3000390611AEF9D739C010F03BAE119E1350F4
:100A400012003D3D3D3D3D3D3D3D3D3D3D3D3D3D3E
:100A50003D3D3D3D3D3D3D3D3D3D3D3D3D3D3D3DC6
:100A60003D3D3D3D3D3D3D3D3D004E657720435084
:100A70005520636869702064657465637465642ECD
:100A800000003D3D3D3D3D3D3D3D3D3D3D3D3D3D10
:100A90003D3D3D3D3D3D3D3D3D3D3D3D3D3D3D3D86
:100AA0003D3D3D3D3D3D3D3D3D003D3D3D3D3D3DB3
:100AB0003D3D3D3D3D3D3D3D3D3D3D3D3D3D3D3D66
:100AC0003D3D3D3D3D3D3D3D3D3D3D3D3D3D3D3D56
:100AD0003D0053696572726120526164696F2053F1
:100AE000797374656D732054522053657175656E0A
:100AF000636572004669726D776172652076657212
:100B000073696F6E20002C206275696C6420000090
:100B10004E6574776F726B206164647265737320C5
:100B20002000456E746572202F2F68656C702066FA
:100B30006F7220636F6D6D616E642073756D6D6192
:100B4000727900003D3D3D3D3D3D3D3D3D3D3D3DDE
:100B50003D3D3D3D3D3D3D3D3D3D3D3D3D3D3D3DC5
:100B60003D3D3D3D3D3D3D3D3D3D3D00456E74655A
:100B70007220636F6D6D616E642000002F2F6F75A2
:100B8000743033206F6E00004641494C00004865C8
:100B90007921206E657720636F6D6D616E64000052
:100BA0006E65745F7061636B65742073686F756CDC
:100BB0006420626520636C656172203C00006E6594
:100BC000745F7061636B65745F6C656E203D2000BF
:100BD0007061636B6574203D20006E65745F73798E
:100BE0006E633D006E65745F747970653D006E657F
:100BF000745F66726F6D3D006E65745F746F3D006B
:100C00006E65745F6372633D00006E65745F706152
:100C1000796C6F61643D3C006E65745F7061636BFD
:100C200065745F6C656E3D006E65745F7061796CB4
:100C30006F61645F6C656E3D00002E2E2E20636830
:100C400065636B2074686520435243202E2E2E006E
:100C50006C656E677468206F6620617267203D2046
:100C6000000043616C63756C61746564204352439A
:100C7000203D20002C205061636B6574204352435B
:100C8000203D2000435243204661696C65642E205C
:100C900020426164207061636B657400435243209D
:100CA00050617373656420212020476F6F6420506A
:100CB00061636B6574006D79206164647265737340
:100CC0003D00484559212074686973207061636B49
:100CD000657420697320666F72206D6521004E6F08
:100CE00074206D79206164647265737300005365CC
:100CF0006E643A20000053656E643A20000053652C
:100D00006E643A20000053656E643A20000049206A
:100D10006861766520746865206E6574776F726BA4
:100D200020286E65745F61737365727420616374EB
:100D30006976652900004E6574776F726B20726565
:100D40006C656173656400004E6F77206174207478
:100D5000686520657865637574655F6E65745F634B
:100D60006F6D6D616E642073746570006E65745F85
:100D70007061636B65745F6C656E3D3D00002020A3
:100D8000636D645F64656C696D3D3D002020636D3B
:100D9000645F64656C696D3D3D3D0000636D645F3B
:100DA00064656C696D20203D0000636D645F636F56
:100DB0006D6D616E643D0000636D645F61726720FC
:100DC0002020203D00004F4E44454C415931000049
:100DD0004F4E44454C41593200004F4E44454C4122
:100DE000593300004F4E44454C41593400004F4E9A
:100DF00044454C41593500004F464644454C415905
:100E000031004F464644454C415932004F46464416
:100E1000454C415933004F464644454C41593400F6
:100E20004F464644454C41593500454E41424C459C
:100E3000000044495341424C45004E4F524D414CF5
:100E40004F4E00004F6E2073657175656E636520AF
:100E50003D206E6F726D616C0000524556455253D5
:100E6000454F4E004F6E2073657175656E6365204A
:100E70003D2072657665727365004E4F524D414C50
:100E80004F4646004F66662073657175656E6365F3
:100E9000203D206E6F726D616C0052455645525375
:100EA000454F464600004F66662073657175656E56
:100EB0006365203D207265766572736500004F554D
:100EC000543031004F55543032004F5554303300B8
:100ED0004F55543034004F5554303500494E310091
:100EE000494E3200494E330050554C53450043574C
:100EF00000004B455945520057504D00574D0000DA
:100F0000574D4C494D4954004144314D494E000024
:100F10004144324D494E00004144334D494E00009A
:100F20004144344D494E00004144314D4158000088
:100F30004144324D415800004144334D4158000076
:100F40004144344D415800004144414C41524D0010
:100F5000414443414C310000414443414C32000084
:100F6000414443414C330000414443414C34000070
:100F700053455452455600005345544255494C443C
:100F800000004E4554004C4F43414C0048454C50E6
:100F900000004C4F4144000053415645000053545B
:100FA0004154555300005354415445004445425563
:100FB000474F4E004465627567206D6F6465204F32
:100FC0004E0044454255474F464600004465627511
:100FD00067206D6F6465204F4646000053524445BC
:100FE0004255474F4E0053686966742072656769C1
:100FF00073746572206465627567206D6F64652027
:101000004F4E0000535244454255474F464600005C
:1010100053686966742072656769737465722064C9
:1010200065627567206D6F6465204F4646004E45CA
:101030005444454255474F4E00004E6574776F72D9
:101040006B206465627567206D6F6465204F4E008C
:101050004E455444454255474F4646004E657477C9
:101060006F726B206465627567206D6F6465204FD9
:101070004646000050494E470000524F4C4C4341F9
:101080004C4C0000464F5243454641494C0045599F
:101090004543414E44590000455945004D5347448E
:1010A000495245435400536574206D6573736167FD
:1010B00065206D6F646520746F2064697265637468
:1010C0002E004D53474E45540000536574206D6506
:1010D0007373616765206D6F646520746F206E6542
:1010E00074776F726B207061636B6574206D6F64D1
:1010F000652E00004543484F000053544154455469
:101100005249474745520000524553455400524505
:10111000424F4F5400004745544144445200534508
:101120005441444452005241440053494C454E54AA
:1011300000004D4F44450000424F4F5400002050E6
:10114000494E473A20002C2046726F6D3A2000002D
:101150002C20416464726573733A200053544154E7
:1011600045313A005354415445313A0053544154A7
:1011700045313A005354415445323A005354415496
:1011800045333A005354415445343A005354415482
:1011900045353A005354415445313A005354415473
:1011A00045323A005354415445333A005354415464
:1011B00045343A005354415445353A004F4B0000F2
:1011C00053595354454D204641494C2C2066726F6B
:1011D0006D3A20002E20205368757474696E672064
:1011E000646F776E2E0053657420504320757064D1
:1011F000617465207472696767657220746F20007E
:101200004F4E00004B65796572206D6F6465204F0D
:101210004E004B65796572206D6F6465204F4646C0
:101220000000536574204357207370656564207413
:101230006F20000053656E642043573A20002D2D27
:101240002D2D2D20412F4420434F4E5645525445BD
:10125000522056414C554553202D2D2D2D2D2D2DF1
:101260002D2D0000416E616C6F6720696E2031206A
:101270003D20000076202046776420202800416E23
:10128000616C6F6720696E2032203D20000076205F
:101290002052656620202800416E616C6F672069CE
:1012A0006E2033203D2000007620202020202020AA
:1012B0002800416E616C6F6720696E2034203D20EC
:1012C0000000762020202020202028002D2D2D2DEC
:1012D0002D2D2D2D2D2D2D2D2D2D2D2D2D2D2D2D3E
:1012E0002D2D2D2D2D2D2D2D2D2D2D2D2D2D2D2D2E
:1012F00000004F4E0000416E616C6F6720696E7098
:10130000757420616C61726D206D6F6465204F4E45
:1013100000004F464600416E616C6F6720696E7039
:10132000757420616C61726D206D6F6465204F462D
:10133000460053657420412F442031206D696E6949
:101340006D756D20746F200053657420412F44200B
:1013500032206D696E696D756D20746F2000536564
:101360007420412F442033206D696E696D756D20A6
:10137000746F200053657420412F442034206D6920
:101380006E696D756D20746F200053657420412F58
:10139000442031206D6178696D756D20746F200077
:1013A00053657420412F442032206D6178696D753A
:1013B0006D20746F200053657420412F442033202A
:1013C0006D6178696D756D20746F200053657420B0
:1013D000412F442034206D6178696D756D20746FE4
:1013E000200053657420412F4420696E707574206D
:1013F000312063616C6962726174696F6E2076611D
:101400006C756520746F200053657420412F442053
:10141000696E70757420322063616C6962726174E8
:10142000696F6E2076616C756520746F200053655E
:101430007420412F4420696E7075742033206361DD
:101440006C6962726174696F6E2076616C7565207B
:10145000746F200053657420412F4420696E7075AD
:101460007420342063616C6962726174696F6E20EC
:1014700076616C756520746F2000212121204C6FEE
:101480007720766F6C7461676520616C61726D2086
:101490006F6E20696E7075742023302E20204D6988
:1014A0006E203D200000762E202041637475616C13
:1014B000203D2000212121204C6F7720766F6C7415
:1014C00061676520616C61726D206F6E20696E705E
:1014D00075742023312E20204D696E203D200000A0
:1014E000762E202041637475616C203D20002121FF
:1014F00021204C6F7720766F6C7461676520616C7A
:1015000061726D206F6E20696E7075742023322EAB
:1015100020204D696E203D200000762E2020416362
:101520007475616C203D2000212121204C6F7720B3
:10153000766F6C7461676520616C61726D206F6E8F
:1015400020696E7075742023332E20204D696E2023
:101550003D200000762E202041637475616C203D93
:101560002000212121204F76657220766F6C7461F6
:10157000676520616C61726D206F6E20696E707599
:10158000742023302E20204D6178203D2000762EBF
:10159000202041637475616C203D200021212120B1
:1015A0004F76657220766F6C7461676520616C613F
:1015B000726D206F6E20696E7075742023312E203D
:1015C000204D6178203D2000762E202041637475E7
:1015D000616C203D2000212121204F76657220760C
:1015E0006F6C7461676520616C61726D206F6E2035
:1015F000696E7075742023322E20204D6178203D55
:101600002000762E202041637475616C203D2000FF
:10161000212121204F76657220766F6C7461676599
:1016200020616C61726D206F6E20696E7075742020
:1016300023332E20204D6178203D2000762E20205F
:1016400041637475616C203D20004F464600576130
:101650007474206D657465722070726F7465637444
:10166000696F6E2064697361626C656400004F4E3F
:10167000000042617369632077617474206D657442
:1016800065722070726F74656374696F6E20656E29
:1016900061626C656400435553544F4D0000456EC4
:1016A00061626C65207573657220646566696E653C
:1016B000642077617474206D657465722070726F38
:1016C00074656374696F6E2072616E6765004B6547
:1016D0007920696E70757420676F657320696E611B
:1016E0006374697665004B657920696E7075742046
:1016F000676F6573206163746976650053494C4573
:101700004E540000564552424F534500426F6F748D
:1017100020696E20766572626F7365206D6F6465F7
:1017200000004F4E000053696C656E74206D6F644D
:1017300065204F4646004C4F43414C004E455457A0
:101740004F524B0043616C6C207369676E20736568
:101750007420746F2000536574206669726D776120
:1017600072652072657620746F20000053657420C6
:101770006669726D77617265206275696C64207448
:101780006F2000004E6574776F726B206164647225
:101790006573732073657420746F20005365742023
:1017A0006D79206E6574776F726B20616464726509
:1017B000737320746F200000536574205478204F99
:1017C0004E2064656C6179203120746F2000536570
:1017D00074205478204F4E2064656C61792032204B
:1017E000746F2000536574205478204F4E20646538
:1017F0006C6179203320746F200053657420547815
:10180000204F4E2064656C6179203420746F200075
:10181000536574205478204F4E2064656C617920A4
:101820003520746F20005365742052782064656CF5
:101830006179203120746F20000053657420527844
:101840002064656C6179203220746F20000053653C
:10185000742052782064656C6179203320746F2085
:1018600000005365742052782064656C61792034DF
:1018700020746F2000005365742052782064656CDA
:101880006179203520746F2000004F757470757475
:10189000200020656E61626C656400004F75747095
:1018A000757420002064697361626C6564004F4E3A
:1018B00000004F4646005475726E206F7574707547
:1018C000742031204F4E00005475726E206F757475
:1018D0007075742031204F4646004F4E00004F4631
:1018E00046005475726E206F7574707574203220C6
:1018F0004F4E00005475726E206F757470757420B1
:1019000032204F4646004F4E00004F464600547569
:10191000726E206F75747075742033204F4E000006
:101920005475726E206F75747075742033204F4635
:1019300046004F4E00004F4646005475726E206FB1
:1019400075747075742034204F4E00005475726E9B
:10195000206F75747075742034204F4646004F4ECA
:1019600000004F4646005475726E206F7574707596
:10197000742035204F4E00005475726E206F7574C0
:101980007075742035204F4646004F4E00004F467C
:1019900046005475726E20696E7075742031204F48
:1019A0004E005475726E20696E7075742031204F30
:1019B000464600004F4E00004F4646005475726E7A
:1019C00020696E7075742032204F4E005475726E0F
:1019D00020696E7075742032204F464600004F4ECD
:1019E00000004F4646005475726E20696E70757423
:1019F0002033204F4E005475726E20696E707574DE
:101A00002033204F46460000526573657420616C98
:101A10006C20706172616D657465727320746F20E3
:101A200064656661756C742076616C7565732E00F3
:101A3000436F6E66696775726174696F6E2073615A
:101A400076656420746F20666C617368206D656DC7
:101A50006F72792E0000436F6E66696775726174EC
:101A6000696F6E206C6F616465642066726F6D20B3
:101A7000666C617368206D656D6F72792E002D2D17
:101A80002D20545220537175656E63657220436F2B
:101A90006D6D616E6473202D2D2D2D2D2D2D2D2D11
:101AA0002D2D2D2D2D2D2D2D2D2D2D2D2D2D2D2D66
:101AB0002D2D2D2D2D2D2D2D2D004F4E44454C41DE
:101AC00059306E207820206D732E2044656C61792A
:101AD00020782028312D3530303029206D732E208C
:101AE0006265666F7265207475726E696E67206FCD
:101AF0006E206F757470757420236E2C20207768AB
:101B0000657265206E203D20312D35004F464644DC
:101B1000454C4159306E2078206D732E2044656C01
:101B2000617920782028312D3530303029206D73AF
:101B30002E206265666F7265207475726E696E67BD
:101B4000206F6666206F757470757420236E2C206C
:101B50007768657265206E203D20312D35004E4F2F
:101B6000524D414C4F4E2020202020202020205438
:101B700075726E206F6E2020696E206E6F726D61BF
:101B80006C202073657175656E63652C20312C2087
:101B9000322C20332C20342C20352020284465661C
:101BA00061756C7429004E4F524D414C4F46462092
:101BB000202020202020205475726E206F66662021
:101BC000696E206E6F726D616C2020736571756532
:101BD0006E63652C20352C20342C20332C20322CA5
:101BE000203120202844656661756C7429005245B7
:101BF00056455253454F4E2020202020202020546F
:101C000075726E206F6E2020696E20726576657227
:101C100073652073657175656E63652C20352C20A6
:101C2000342C20332C20322C2031000052455645D4
:101C30005253454F464620202020202020547572C4
:101C40006E206F666620696E2072657665727365B8
:101C50002073657175656E63652C20312C20322CE4
:101C600020332C20342C20350000454E41424C4579
:101C70002078202020202020202020456E61626CCA
:101C80006573206F757470757420782028312D3538
:101C9000290044495341424C4520782020202020EF
:101CA00020202044697361626C6573206F757470C5
:101CB000757420782028312D352900002D2D2D20F8
:101CC00041646D696E20436F6D6D616E6473202D8C
:101CD0002D2D2D2D2D2D2D2D2D2D2D2D2D2D2D2D34
:101CE0002D2D2D2D2D2D2D2D2D2D2D2D2D2D2D2D24
:101CF0002D2D2D2D2D2D2D2D000048454C50202013
:101D00002020202020202020202020446973706C77
:101D1000617920746869732068656C7020696E66EB
:101D20006F726D6174696F6E000053544154555366
:101D30002020202020202020202020446973706C47
:101D40006179207468652063757272656E742063B2
:101D50006F6E66696775726174696F6E00004C4FD3
:101D60004144202020202020202020202020204C02
:101D70006F616420636F6E66696775726174696F05
:101D80006E2066726F6D20666C617368206D656D84
:101D90006F727900534156452020202020202020BA
:101DA00020202020205361766520636F6E6669676E
:101DB00075726174696F6E20746F20666C617368F0
:101DC000206D656D6F727900524553455420202077
:101DD0002020202020202020205265736574206F51
:101DE0007065726174696E6720706172616D65748F
:101DF00065727320746F207374616E646172642005
:101E000064656661756C742076616C75657300003D
:101E10005245424F4F5420202020202020202020B7
:101E2000205265626F6F74207468652073797374D3
:101E3000656D0000424F4F542053494C454E54208D
:101E400020202020205475726E73206F66662062F9
:101E50006F6F74206D65737361676500424F4F54F7
:101E600020564552424F5345202020202054757261
:101E70006E73206F6E20626F6F74206D6573736177
:101E800067650000535441544554524947474552F1
:101E900020787878205570646174657320504320F1
:101EA00070726F6772616D20646973706C61792004
:101EB00069662064656C6179206973203E207878BA
:101EC00078202864656661756C74203D2032353059
:101ED000206D732900002D2D2D20412F4420436FAC
:101EE0006E766572746572202D20416E616C6F672D
:101EF00020496E7075742043616C69627261746907
:101F00006F6E2D2D2D2D2D2D2D2D2D2D2D2D2D2D7E
:101F10002D2D0000414443414C6E207878782020DC
:101F20002020202020416473206F7220737562741A
:101F3000726163747320746865206F66667365747C
:101F4000207878782028696E206D696C69766F6CCE
:101F500074732920746F2074686520412F442063B6
:101F60006F6E76657274657220276E272020283187
:101F70002D34290041446E4D494E20787878202038
:101F8000202020202053657473206C6F772074729A
:101F9000696767657220616C61726D20766F6C7421
:101FA00061676520746F2078787820766F6C747321
:101FB0002028696E20766F6C7473290041446E4D41
:101FC00041582078787820202020202020536574E4
:101FD0007320686967682074726967676572206139
:101FE0006C61726D20766F6C7461676520746F2010
:101FF00078787820766F6C74732028696E20766FFD
:102000006C7473290000524144202020202020209D
:10201000202020202020205265616420616E616CA8
:102020006F6720696E70757420766F6C7461676578
:10203000206E6F7700002D2D2D2057617474204D78
:102040006574657220436F6D6D616E6473202D2D14
:102050002D2D2D2D2D2D2D2D2D2D2D2D2D2D2D2DB0
:102060002D2D2D2D2D2D2D2D2D2D2D2D2D2D2D2DA0
:102070002D2D0000574D204F4E20202020202020C5
:1020800020202020205475726E206F6E20626173B4
:1020900069632077617474206D65746572206D6F5B
:1020A0006E69746F72696E672E20204869676820B8
:1020B0007265666C656374656420706F7765722005
:1020C00064697361626C65732073657175656E63B5
:1020D00065720000574D204F4646202020202020CA
:1020E00020202020205475726E206F666620626169
:1020F0007369632077617474206D65746572206DF7
:102100006F6E69746F72696E672E0000574D2043C1
:102110005553544F4D2020202020202020547572EC
:102120006E206F6E2077617474206D657465722007
:102130006D6F6E69746F72696E672E2020496E68CC
:10214000696269742073657175656E63652077686F
:10215000656E207265666C656374656420766F6C6D
:102160007461676520686974732074686520574DD1
:102170004C494D49542076616C756500574D4C496A
:102180004D4954207878782020202020204D696EF9
:10219000696D756D207265666C6563746564207623
:1021A0006F6C7461676520746861742077696C6C0A
:1021B00020696E686962697420746865207365714E
:1021C00075656E6365002D2D2D20435720436F6D7F
:1021D0006D616E6473202D2D2D2D2D2D2D2D2D2D0A
:1021E0002D2D2D2D2D2D2D2D2D2D2D2D2D2D2D2D1F
:1021F0002D2D2D2D2D2D2D2D2D2D2D2D2D2D2D2D0F
:102200002D2D00004B45594552204F4E20202020B7
:1022100020202020205475726E206F6E206B65790F
:102220006572206D6F64652E20204F757470757413
:1022300020352077696C6C2073656E6420435720CD
:102240007573696E672074686520435720636F6DEE
:102250006D616E6400004B45594552204F46462043
:10226000202020202020205475726E206F6666206A
:102270006B65796572206D6F64652E20204F7574D3
:1022800070757420352077696C6C206F7065726191
:10229000746520696E206E6F726D616C207365715C
:1022A00075656E636572206D6F64650043572078B5
:1022B0007878787820202020202020202053656EF8
:1022C00064207465787420787878787820696E2036
:1022D0004357207573696E67206F7574707574202D
:1022E0003520696E206B65796572206D6F646500BD
:1022F00057504D207878202020202020202020209A
:102300002053657420435720737065656420696E9F
:1023100020617070726F78696D61746520776F727B
:10232000647320706572206D696E75746520283144
:102330002D39392900002D2D2D204E6574776F72AF
:102340006B20436F6D6D616E6473202D2D2D2D2DCF
:102350002D2D2D2D2D2D2D2D2D2D2D2D2D2D2D2DAD
:102360002D2D2D2D2D2D2D2D2D2D2D2D2D2D2D2D9D
:102370002D2D0000534554414444522078782020AC
:1023800020202020205768657265207878206973A6
:102390002074686520626F6172642773206E6574B3
:1023A000776F726B20616464726573732028626555
:1023B000747765656E203120616E642031352900A7
:1023C00047455441444452202020202020202020F2
:1023D00020476574207468652076616C7565206F90
:1023E000662074686520626F6172642773206E6571
:1023F00074776F726B206164647265737300534904
:102400004C454E54204F4E20202020202020204498
:102410006F206E6F742073656E64206D65737361D9
:1024200067657320746F2073657269616C20706FCB
:102430007274207768656E207374617465206368B8
:10244000616E6765730053494C454E54204F4646B4
:102450002020202020202053656E64206D6573733A
:102460006167657320746F2073657269616C207099
:102470006F7274207768656E207374617465206371
:1024800068616E67657300004D5347444952454388
:102490005420202020202020205365742072657352
:1024A000706F6E736520746F20706C61696E20743C
:1024B00065787420666F726D617400004D53474EED
:1024C00045542020202020202020202020536574E7
:1024D00020726573706F6E736520746F206E657403
:1024E000776F726B207061636B657420666F726DBD
:1024F000617400002D2D2D204D616E75616C204F93
:10250000757470757420436F6D6D616E6473202DEA
:102510002D2D2D2D2D2D2D2D2D2D2D2D2D2D2D2DEB
:102520002D2D2D2D2D2D2D2D2D2D2D2D2D2D2D2DDB
:1025300000004F5554306E204F4E20202020202088
:102540002020204D616E75616C6C79207475726EFF
:10255000204F4E20206F7574707574206E202831C6
:102560002D3529004F5554306E204F4646202020EF
:1025700020202020204D616E75616C6C792074756F
:10258000726E204F4646206F7574707574206E20F1
:1025900028312D3529002D2D2D20496E7465726E40
:1025A000616C20446562756767696E6720436F6D73
:1025B0006D616E6473202D2D2D2D2D2D2D2D2D2D26
:1025C0002D2D2D2D2D2D2D2D2D2D2D2D2D2D2D2D3B
:1025D0002D2D000044454255474F4E2020202020FD
:1025E00020202020205475726E206F6E206465625A
:1025F000756767696E67206D6573736167657300E2
:1026000044454255474F4646202020202020202088
:10261000205475726E206F66662064656275676708
:10262000696E67206D657373616765730000464F5F
:102630005243454641494C2020202020202020465E
:102640006F7263657320756E697420696E746F2094
:102650004641494C206D6F64652E20205368757487
:1026600073206F666620616C6C206F757470757472
:1026700073003D3D3D3D3D5B2043555252454E5418
:1026800020434F4E46494755524154494F4E205DD5
:102690003D3D3D3D3D3D3D3D3D00436F6E666967BF
:1026A00020636F646520203A2000426F61726420CD
:1026B000747970652020203A200046572076657294
:1026C00073696F6E2020203A20004657206275699A
:1026D0006C6420202020203A20004D792061646421
:1026E000726573732020203A20004F4E20206465CD
:1026F0006C6179203120203A20004F4E2020646503
:102700006C6179203220203A20004F4E20206465F1
:102710006C6179203320203A20004F4E20206465E0
:102720006C6179203420203A20004F4E20206465CF
:102730006C6179203520203A20004F4646206465A0
:102740006C6179203120203A20004F464620646594
:102750006C6179203220203A20004F464620646583
:102760006C6179203320203A20004F464620646572
:102770006C6179203420203A20004F464620646561
:102780006C6179203520203A20003A20456E616244
:102790006C6564003A2044495341424C4544000072
:1027A0004F757470757420312020202020003A204D
:1027B000456E61626C6564003A2044495341424C65
:1027C000454400004F75747075742032202020201D
:1027D00020003A20456E61626C6564003A204449ED
:1027E0005341424C454400004F757470757420335A
:1027F0002020202020003A20456E61626C65640034
:102800003A2044495341424C454400004F7574708E
:10281000757420342020202020003A20456E61620B
:102820006C6564003A2044495341424C45440000E1
:102830004F757470757420352020202020004F4E75
:102840002073657175656E636520203A204E6F7246
:102850006D616C004F4E2073657175656E63652008
:10286000203A205265766572736564004F464620B3
:1028700073657175656E6365203A204E6F726D6188
:102880006C004F46462073657175656E6365203A2E
:1028900020526576657273656400435720737065D6
:1028A000656420202020203A200057617474206D38
:1028B0006574657220636865636B696E67204F4657
:1028C000460053696D706C652077617474206D6586
:1028D00074657220636865636B696E6720656E61FD
:1028E000626C6564000057617474206D6574657274
:1028F000206C696D69742073657420746F2000000A
:10290000414420616C61726D206D6F64653A204FA7
:1029100066660000414420616C61726D206D6F64D9
:10292000653A204F4E00416E616C6F672031206D1B
:10293000696E203A20002020202020202020206DB9
:102940006178203A200020202020202020202063B1
:10295000616C203A2000416E616C6F672032206DFF
:10296000696E203A20002020202020202020206D89
:102970006178203A20002020202020202020206381
:10298000616C203A2000416E616C6F672033206DCE
:10299000696E203A20002020202020202020206D59
:1029A0006178203A20002020202020202020206351
:1029B000616C203A2000416E616C6F672034206D9D
:1029C000696E203A20002020202020202020206D29
:1029D0006178203A20002020202020202020206321
:1029E000616C203A2000436F6D6D206D6F6465202F
:1029F0002020203A204C6F63616C0000436F6D6DA6
:102A0000206D6F6465202020203A204E6574776F1A
:102A1000726B0000F86A400E386E006A030EAF6EEB
:102A2000200EAC6E900EAB6E2EEE81F094988298D4
:102A3000949A829A939081909392819293948194A4
:102A4000110E05012E6FC70E2D6F510E2C6F810ECA
:102A50002B6F0101D99DD98F040E196EB00E186E1F
:102A60001D6A90C51CF09CEC02F005018E6F19C028
:102A70008FF5030E8D6F520E8C6F05EEDCF0540E49
:102A8000EE6E520EEE6E310EEE6EEF6A000180EFCA
:102A900015F09EAA23D0060EAB141DE1E2CF3DF047
:102AA000E1CF3CF03E2AFF0E3E5C01E33E6A1DEEA4
:102AB00082F03E50E126000EE222AECFE7FF0D0E7F
:102AC000E75C02E1010E426E3EC017F43DC0E2FF3A
:102AD0003CC0E1FF1100AB98AB8800D011003E6A0A
:102AE0003F6A9D8AC00EF26E12009D9A0DEE82F032
:102AF000FF0EEE6AE82EFDD73E6A3F6A9D8A1200FD
:102B0000400EAF6E900EAB6E200EAC6E0B0EC16E13
:102B1000F19E320E24EC02F08298829A819081928A
:102B20008194939481949392819293908190949ABA
:102B3000829A949882980101D99BD9BF8282D9AF99
:102B4000829205012A910101CC6BD46BDB6BDA6BAD
:102B500001EEDCF04F0EEE6E4B0EEE6EEF6A01EE04
:102B60001CF0EE6A01EEE1F0EE6A0401A06B640E67
:102B70009F6FA26BA16B04EE19F0300EEE6EEE6E3D
:102B8000EF6A06010989098B099D0401A36B04EE14
:102B9000A4F0EE6A0501276B266BE689E68BE68DCD
:102BA000E68F0601098109930501776BCD0E7B6FD6
:102BB000CC0E7A6F4C0E796F7C0E786F06010995FA
:102BC00009970101686B6A6B0501256B4A6B496BBC
:102BD000486B476B4E6B4D6B4C6B4B6B526B516B39
:102BE000506B4F6B566B556B546B536B01016B6B9A
:102BF00005015A6B596B586B576B5E6B5D6B5C6B69
:102C00005B6B626B616B606B5F6B666B656B646B60
:102C1000636B6A6B696B700E686F830E676F6E6BA8
:102C20006D6B700E6C6F830E6B6F726B716B700ED1
:102C3000706F830E6F6F766B756B700E746F830E93
:102C4000736F01016C6B4BDF00012DEC18F001017B
:102C5000D991D993D995010E0501E36F010ED76F74
:102C6000D96B040ED86FDB6B220EDA6F010EE56FA5
:102C70005A6B596B586B576B6A6B696B200E686F98
:102C8000810E676F5E6B5D6B5C6B5B6B6E6B6D6B10
:102C9000200E6C6F810E6B6F626B616B606B5F6B94
:102CA000726B716B200E706F810E6F6F666B656B50
:102CB000646B636B766B756B200E746F810E736F34
:102CC000E697296B640E286FE329E46F0001D5ECC9
:102CD00029F082B66DEF16F0F9D794908280000E3D
:102CE000F5EC01F00501D76FD7290001D8A4A4EFB6
:102CF00016F00401A3530001D8A4A4EF16F004EECB
:102D0000A4F00A0EF76E420EF66ED9EC02F0EF6AEE
:102D100028EC1EF004EEA4F00A0EF76E6A0EF66EB2
:102D2000D9EC02F0EF6A28EC1EF025EC43F0C4EC7D
:102D300043F004EEA4F00A0EF76E820EF66ED9ECA4
:102D400002F0EF6A28EC1EF0E3EC46F00AEC38F0F3
:102D500001EE6DF0020E016E0501E551CCEC00F0C4
:102D6000EF6A010E0401A353D8A4000E356E010EC4
:102D700001016B53D8A4000E35140001D8B436EF0E
:102D800017F004EEA4F00A0EF76EAA0EF66ED9EC58
:102D900002F0EF6A28EC1EF004EEA4F00A0EF76EC3
:102DA000D20EF66ED9EC02F0EF6A28EC1EF004EEBB
:102DB000A4F00A0EF76EF40EF66ED9EC02F0020ED5
:102DC000016E086AD9C521F0D8C520F0CFEC00F01B
:102DD0000B0EF76E060EF66ED9EC02F0020E016EC7
:102DE000086ADBC521F0DAC520F0CFEC00F0EF6A0D
:102DF00028EC1EF004EEA4F00B0EF76E100EF66E2B
:102E0000D9EC02F0020E016E0501E551CCEC00F0A8
:102E1000EF6A04EEA4F00B0EF76E220EF66ED9ECFC
:102E200002F0EF6A000128EC1EF004EEA4F00B0E95
:102E3000F76E440EF66ED9EC02F0EF6A28EC1EF045
:102E400004EEA4F00B0EF76E6C0EF66ED9EC02F0E9
:102E5000EF6A28EC1EF004EEA4F00B0EF76E7C0E69
:102E6000F66ED9EC02F0EF6A0EEC1EF0320E24EC96
:102E700002F0949082900B0EF76E880EF66E01EEC3
:102E8000DCF001EC03F0D8A448EF17F036EC2AF0A0
:102E9000D896060109ADD8860001D8B652EF17F0D2
:102EA00087EF17F001EEA0F0020E016EE86A80BA1B
:102EB000010ECCEC00F0EF6A01EEA0F084EC00F023
:102EC000808AE8A0809A01EEB5F0020E016EE86AF1
:102ED00081B6010ECCEC00F0EF6A01EEB5F084ECA7
:102EE00000F08186E8A081962CEC2FF0010E010104
:102EF0006C5D0001D8A47FEF17F0EEEC34F0050113
:102F000077530001D8B487EF17F095EC37F006013E
:102F1000099D000181A88FEF17F0EDEF17F0010E6A
:102F20000101CC6FE86A80BA010E356EE86A81B69D
:102F3000010E35100001D8B4A3EF17F00101CC6BDE
:102F40000001A6EF17F0010E0101CC6F0001010E88
:102F50000101CC5D010ED8A4000E356E010E0501F5
:102F60002ABDE86A35140001D8B4B9EF17F09DEF17
:102F70003DF0010E0101CC5D010ED8A4000E356EAE
:102F8000E86A05012ABD010E35140001D8B4CBEF63
:102F900017F01BEF38F0010E0101CC53D8A4000E3E
:102FA000356E010E05012ABDE86A35140001D8B45A
:102FB000DCEF17F0DEEF3AF0010E0101CC53D8A49C
:102FC000000E356EE86A05012ABD010E35140001B8
:102FD000D8B4EDEF17F0A2EF3DF00501264B272BFB
:102FE0002651285D275129590001D8B016EF18F055
:102FF0000501276B266BD8962AB1D8860001D8B672
:1030000009EF18F005012A8194928292000116EFCF
:1030100018F0D89605012AA1D8860001D8B615EF78
:1030200018F005012A919492828200010401A151B5
:103030009F5DA251A0590001D8B024EF18F02DECEB
:1030400018F00401A26BA16B0001010E425CD8A430
:103050002CEF18F031EC18F00ED7426A75EC15F031
:103060001200D8960101D9A5D8860001D8B645EF3F
:1030700018F00B0EF76E8E0EF66ED7EC01F00D0EFB
:10308000DFEC01F00A0EDFEC01F001EEE1F0820E60
:10309000EE6AE82EFDD7D8960101D9A5D8860001A1
:1030A000D8B669EF18F00B0EF76EA00EF66ED7ECDF
:1030B00001F001EEE1F0EE5003E0DFEC01F0FBD7B0
:1030C0003E0EDFEC01F00D0EDFEC01F00A0EDFEC3E
:1030D00001F03E040401176F00013EAE72EF18F0DC
:1030E0000401176B0001D8960101D9A5D88600010B
:1030F000D8B68DEF18F00B0EF76EBE0EF66ED7EC4D
:1031000001F0040E016E04011751CCEC00F00D0E1D
:10311000DFEC01F00A0EDFEC01F0000104011753AF
:103120000001D8A497EF18F0010E0401176F0001F9
:10313000040117050B6E0101CC6B00010101CC519C
:103140000B5C0001D8A0DDEF18F0D8960101CCAFE0
:10315000D8860001D8B6AFEF18F00101CC6B0001A2
:103160000101CC290DEE82F0E926000EEA22EFCF14
:103170000FF001EEE1F0CC51E926000EEA220FC07B
:10318000EFFFD896D9A5D8860001D8B6D7EF18F0AA
:10319000040E016E01EEE1F00101CC51E926000EB2
:1031A000EA22EF50CCEC00F0200EDFEC01F0000141
:1031B0000101CC2B0001D8A4C0D7E0EC18F012001C
:1031C00001EEE1F011EEE1F0F5EC02F0D89601012C
:1031D000D9A5D8860001D8B601EF19F00B0EF76E0D
:1031E000D00EF66ED7EC01F001EEE1F0EE5003E008
:1031F000DFEC01F0FBD70D0EDFEC01F00A0EDFEC87
:1032000001F002EE63F011EEE1F0010EF36E010E3B
:10321000E1EC02F0EF6AD8960101D9A5D886000149
:10322000D8B626EF19F00B0EF76EDA0EF66ED7EC65
:1032300001F002EE63F0EE5003E0DFEC01F0FBD7AB
:103240000D0EDFEC01F00A0EDFEC01F002EE65F08E
:1032500011EEE1F0020EF36E010EE1EC02F0EF6A06
:10326000D8960101D9A5D8860001D8B64BEF19F040
:103270000B0EF76EE40EF66ED7EC01F002EE65F081
:10328000EE5003E0DFEC01F0FBD70D0EDFEC01F0B8
:103290000A0EDFEC01F002EE68F011EEE1F0030E31
:1032A000F36E020EE1EC02F0EF6AD8960101D9A5A7
:1032B000D8860001D8B670EF19F00B0EF76EEE0E3F
:1032C000F66ED7EC01F002EE68F0EE5003E0DFECB2
:1032D00001F0FBD70D0EDFEC01F00A0EDFEC01F080
:1032E00002EE6CF011EEE1F0050EF36E020EE1EC71
:1032F00002F0EF6AD8960101D9A5D8860001D8B6A8
:1033000095EF19F00B0EF76EF80EF66ED7EC01F094
:1033100002EE6CF0EE5003E0DFEC01F0FBD70D0E97
:10332000DFEC01F00A0EDFEC01F002EE70F011EEBE
:10333000E1F0070EF36E030EE1EC02F0EF6AD896AF
:103340000101D9A5D8860001D8B6BAEF19F00C0E44
:10335000F76E000EF66ED7EC01F002EE70F0EE5054
:1033600003E0DFEC01F0FBD70D0EDFEC01F00A0EFD
:10337000DFEC01F002EE75F011EEE1F00A0EF36EF3
:10338000090E0401175DE1EC02F0EF6AD896010125
:10339000D9A5D8860001D8B6E4EF19F00C0EF76E67
:1033A0000A0EF66ED7EC01F002EE75F0EE5003E077
:1033B000DFEC01F0FBD73E0EDFEC01F00D0EDFEC91
:1033C00001F00A0EDFEC01F001EEE1F0E86AEE52E6
:1033D00002E0E83EFCD70401176FD8960101D9A599
:1033E000D8860001D8B607EF1AF00C0EF76E180E4B
:1033F000F66ED7EC01F0040E016E04011751CCEC0F
:1034000000F00D0EDFEC01F00A0EDFEC01F0000120
:1034100002EE75F0E86AEE5202E0E83EFCD70401E5
:10342000186FD8960101D9A5D8860001D8B62BEF20
:103430001AF00C0EF76E280EF66ED7EC01F0040EA3
:10344000016E04011851CCEC00F00D0EDFEC01F020
:103450000A0EDFEC01F0000104EE19F012EE68F044
:10346000030EE75204E0E6CFEEFFE82EFAD7EF6A4C
:10347000300E0201655D0001D8A441EF1AF0E5EFBE
:103480001BF02F0E0201655D0001D8A44AEF1AF06F
:103490000101D98B00012F0E0201655D0001D8A446
:1034A00057EF1AF004EE19F0300EEE6EEF6A2F0EA1
:1034B0000201655D0001D8A460EF1AF0B2EC1FF0C4
:1034C0002F0E0201655D0001D8A46CEF1AF0010116
:1034D0006A6B00016FEF1AF0010E01016A6F0001C3
:1034E0002F0E0201655D0001D8A478EF1AF01200DA
:1034F000D8960101D9A5D8860001D8B68CEF1AF06C
:103500000C0EF76E3A0EF66ED7EC01F00D0EDFECF6
:1035100001F00A0EDFEC01F0D8960101D9A5D8869A
:103520000001D8B6A6EF1AF00C0EF76E500EF66E2C
:10353000D7EC01F0040E016E0101D451CCEC00F087
:103540000D0EDFEC01F00A0EDFEC01F000010401CA
:10355000166B010E0101CC6F0001060E0101CC5D5E
:103560000001D8B010EF1BF001EEE1F00101CC51E9
:10357000E926000EEA22EF50D46FD4510401161B45
:1035800001EEA0F0020E016E0101CC51CCEC00F076
:10359000EF6A01EEB5F0020E016E04011651CCEC9B
:1035A00000F0EF6AD8960101D9A5D8860001D8B6F7
:1035B0000AEF1BF001EEA0F0EE5003E0DFEC01F0AB
:1035C000FBD7200EDFEC01F001EEE1F00101CC5160
:1035D000E926000EEA22EF50DFEC01F0200EDFECCE
:1035E00001F0630EDFEC01F0720EDFEC01F0630E10
:1035F000DFEC01F03D0EDFEC01F001EEB5F0EE5036
:1036000003E0DFEC01F0FBD70D0EDFEC01F00A0E5A
:10361000DFEC01F000010101CC2B0001D8A49CD704
:10362000090E0101CC6F00010101CC510401175DAD
:103630000001D8A078EF1BF001EEE1F00101CC51C0
:10364000E926000EEA22EF500B6E0B500401161B08
:1036500001EEA0F0020E016E0101CC51CCEC00F0A5
:10366000EF6A01EEB5F0020E016E04011651CCECCA
:1036700000F0EF6AD8960101D9A5D8860001D8B626
:1036800072EF1BF001EEA0F0EE5003E0DFEC01F072
:10369000FBD7200EDFEC01F001EEE1F00101CC518F
:1036A000E926000EEA22EF50DFEC01F0200EDFECFD
:1036B00001F0630EDFEC01F0720EDFEC01F0630E3F
:1036C000DFEC01F03D0EDFEC01F001EEB5F0EE5065
:1036D00003E0DFEC01F0FBD70D0EDFEC01F00A0E8A
:1036E000DFEC01F000010101CC2B0001D8A49BD735
:1036F000D8960101D9A5D8860001D8B69FEF1BF056
:103700000C0EF76E620EF66ED7EC01F0040E016E31
:1037100004011651CCEC00F00C0EF76E740EF66E30
:10372000D7EC01F002EE70F0EE5003E0DFEC01F0B8
:10373000FBD70D0EDFEC01F00A0EDFEC01F000010B
:1037400002EE70F084EC00F00B6E21C00CF022C091
:103750000DF023C00EF00D500E100AE10C500D10AC
:1037600007E10B50040116190001D8B4D1EF1BF08A
:10377000D8960101D9A5D8860001D8B6CCEF1BF0A8
:103780000C0EF76E840EF66ED7EC01F00D0EDFEC2A
:1037900001F00A0EDFEC01F02DEC18F01200E5EF5D
:1037A0001BF0D8960101D9A5D8860001D8B6E5EF5F
:1037B0001BF00C0EF76E9C0EF66ED7EC01F00D0EA2
:1037C000DFEC01F00A0EDFEC01F0D8960101D9A57B
:1037D000D8860001D8B6FFEF1BF00C0EF76EB60EC0
:1037E000F66ED7EC01F0040E016E0501E551CCEC4C
:1037F00000F00D0EDFEC01F00A0EDFEC01F000012D
:1038000002EE6CF084EC00F00101D46FD76BD45160
:103810000501E55D0001D8A411EF1CF0010E0101C6
:10382000D76F0001630E0101D45D0001D8A41CEF25
:103830001CF0010E0101D76F0001630E0101D45D80
:103840000001D8A427EF1CF0020E01016A6F0001ED
:10385000010E0101D75D0001D8A44DEF1CF0D896F0
:103860000101D9A5D8860001D8B643EF1CF00C0E93
:10387000F76EC20EF66ED7EC01F00D0EDFEC01F024
:103880000A0EDFEC01F002EE75F012EE75F0F5ECC9
:1038900002F0C9EC1FF061EF1CF0D8960101D9A528
:1038A000D8860001D8B661EF1CF00C0EF76EDE0E64
:1038B000F66ED7EC01F00D0EDFEC01F00A0EDFEC36
:1038C00001F02DEC18F0120002EECAF011EE31F00A
:1038D000360EE75204E0E6CFEEFFE82EFAD7EF6AA5
:1038E00075EC1CF01DEC1FF0120003EE0CF0820EC4
:1038F000EE6AE82EFDD702EEB7F02F0EEE6EEF6AFD
:1039000002EEBAF0410EEE6EEF6A02EEBDF0020E6C
:10391000016E0501E551CCEC00F0EF6A02EEBDF05E
:10392000E86AEE5202E0E83EFCD70B6E010E0B5C3B
:103930000001D8A4ACEF1CF001EEB5F0300EEE6E35
:1039400012EEBDF0030EE75204E0E6CFEEFFE82EE4
:10395000FAD7EF6AB8EF1CF001EEB5F012EEBDF049
:10396000030EE75204E0E6CFEEFFE82EFAD7EF6A47
:1039700002EEBDF011EEB5F0140EE75204E0E6CF12
:10398000EEFFE82EFAD7EF6A02EEC1F014EE19F05E
:10399000030EE75204E0E6CFEEFFE82EFAD7EF6A17
:1039A00002EEC1F0E86AEE5202E0E83EFCD7010107
:1039B000D46FD4530001D8A4E4EF1CF002EEC1F0A0
:1039C000300EEE6EEE6EEF6A010E0101D45D000165
:1039D000D8A405EF1DF004EEA4F0300EEE6E12EE4A
:1039E000C1F0030EE75204E0E6CFEEFFE82EFAD76F
:1039F000EF6A02EEC1F014EEA4F0800EE75204E08C
:103A0000E6CFEEFFE82EFAD7EF6A020E0101D45D91
:103A10000001D8A412EF1DF002EEC1F0EE50FEE15D
:103A2000ED52EF6A01EE6DF012EEB7F0020EE752C2
:103A300004E0E6CFEEFFE82EFAD712EEBAF0020E5F
:103A4000E75204E0E6CFEEFFE82EFAD712EEBDF023
:103A5000030EE75204E0E6CFEEFFE82EFAD712EEAF
:103A6000C1F0030EE75204E0E6CFEEFFE82EFAD7EE
:103A700012EECAF0410EE75204E0E6CFEEFFE82E68
:103A8000FAD7EF6A01EE6DF0E86AEE5202E0E83E26
:103A9000FCD70101D86FD76B01EE6DF0E86AEE52EA
:103AA00002E0E83EFCD70B6E010ECC6F0001010175
:103AB000CC510B5C0001D8A07AEF1DF001EE6DF047
:103AC0000101CC51EB50D46FD451D71B01EEA0F0C3
:103AD000020E016ECC51CCEC00F0EF6A01EEB5F0B5
:103AE000020E016ED751CCEC00F0EF6ACC2B000136
:103AF000D8A4DCD702EEC5F0020E016E0101D75149
:103B0000CCEC00F0EF6A02EEC5F0E86AEE5202E09B
:103B1000E83EFCD7D46F010ED45D0001D8A4A0EF1D
:103B20001DF004EEA4F0300EEE6EEE6E12EEC5F057
:103B3000040EE75204E0E6CFEEFFE82EFAD7EF6A74
:103B4000020E0101D45D0001D8A4B5EF1DF004EE12
:103B5000A4F0300EEE6E12EEC5F0040EE75204E053
:103B6000E6CFEEFFE82EFAD7EF6A030E0101D45D2F
:103B70000001D8A4C8EF1DF004EEA4F012EEC5F0C9
:103B8000040EE75204E0E6CFEEFFE82EFAD7EF6A24
:103B900002EEC5F014EEA4F0800EE75204E0E6CF8A
:103BA000EEFFE82EFAD7EF6A03EE0CF012EEB7F054
:103BB000020EE75204E0E6CFEEFFE82EFAD712EE4F
:103BC000BAF0020EE75204E0E6CFEEFFE82EFAD795
:103BD00012EEBDF0030EE75204E0E6CFEEFFE82E52
:103BE000FAD712EEC1F0030EE75204E0E6CFEEFF83
:103BF000E82EFAD712EEC5F0040EE75204E0E6CF45
:103C0000EEFFE82EFAD712EECAF0410EE75204E0BA
:103C1000E6CFEEFFE82EFAD7EF6A1200800E026EB2
:103C2000100E096E400E296E540E286E066A056A43
:103C3000200E016E810E076E040E216EA40E82EC22
:103C400001F00D0E93EC01F00A0E93EC01F012005E
:103C500001016A530001D8A476EF1EF052EC1FF068
:103C6000D8960101D9A5D8860001D8B64BEF1EF031
:103C70000C0EF76EEE0EF66ED7EC01F004EEA4F02B
:103C8000EE5003E0DFEC01F0FBD70D0EDFEC01F0AE
:103C90000A0EDFEC01F00401A3530001D8A45EEF8B
:103CA0001EF004EEA4F0EE5003E0DFEC01F0FBD7D1
:103CB0000D0EDFEC01F00A0EDFEC01F0010E040145
:103CC000A35D0001D8A472EF1EF004EEA4F0EE5044
:103CD00003E0DFEC01F0FBD70D0EDFEC01F00A0E84
:103CE000DFEC01F09BEC1FF01CEF1FF0010E010157
:103CF0006A5D0001D8A4C5EF1EF052EC1FF0D89603
:103D00000101D9A5D8860001D8B69AEF1EF00C0E95
:103D1000F76EF60EF66ED7EC01F004EEA4F0EE505E
:103D200003E0DFEC01F0FBD70D0EDFEC01F00A0E33
:103D3000DFEC01F00401A3530001D8A4ADEF1EF0A5
:103D400004EEA4F0EE5003E0DFEC01F0FBD70D0E23
:103D5000DFEC01F00A0EDFEC01F0010E0401A35DBF
:103D60000001D8A4C1EF1EF004EEA4F0EE5003E071
:103D7000DFEC01F0FBD70D0EDFEC01F00A0EDFECFB
:103D800001F09BEC1FF01CEF1FF0020E01016A5DB9
:103D90000001D8A41CEF1FF00501E551320DF3CF4F
:103DA0001CF0F4CF1DF026EC02F0000152EC1FF0E5
:103DB000D8960101D9A5D8860001D8B6F3EF1EF038
:103DC0000C0EF76EFE0EF66ED7EC01F004EEA4F0CA
:103DD000EE5003E0DFEC01F0FBD70D0EDFEC01F05D
:103DE0000A0EDFEC01F00401A3530001D8A406EF92
:103DF0001FF004EEA4F0EE5003E0DFEC01F0FBD77F
:103E00000D0EDFEC01F00A0EDFEC01F0010E0401F3
:103E1000A35D0001D8A41AEF1FF004EEA4F0EE5049
:103E200003E0DFEC01F0FBD70D0EDFEC01F00A0E32
:103E3000DFEC01F09BEC1FF0120052EC1FF0D89663
:103E40000101D9A5D8860001D8B63AEF1FF00D0EB2
:103E5000F76E060EF66ED7EC01F003EE0CF0EE50A6
:103E600003E0DFEC01F0FBD70D0EDFEC01F00A0EF2
:103E7000DFEC01F0D896060109B7D8860001D8B664
:103E80004FEF1FF003EE0CF0EE5003E0DFEC01F01B
:103E9000FBD70D0EDFEC01F00A0EDFEC01F09BEC1E
:103EA0001FF012000101D76B000101EEA0F0020E1D
:103EB000016EE86A82B6010ECCEC00F0EF6A01EE0A
:103EC000A0F084EC00F00101D46F010ED45D00017C
:103ED000D8A46DEF1FF081EF1FF00101D72B050172
:103EE000E5510A0DF3CF1CF0F4CF1DF026EC02F0E3
:103EF000330E0101D75D0001D8A080EF1FF0120042
:103F0000D3D794908280050E24EC02F0D89601015C
:103F1000D9A5D8860001D8B69AEF1FF00D0EF76E1E
:103F20000E0EF66ED7EC01F00D0EDFEC01F00A0E6E
:103F3000DFEC01F0120094908290D8960101D9A58F
:103F4000D8860001D8B6B1EF1FF00D0EF76E360E11
:103F5000F66ED7EC01F00D0EDFEC01F00A0EDFEC8F
:103F600001F01200D8960101D9ABD8860001D8B66D
:103F7000C8EF1FF002EE75F011EEE1F0030EF36EE4
:103F8000000E0401175DE1EC02F0EF6A0101D99B1C
:103F90000001D8960101D9A5D8860001D8B6DDEF79
:103FA0001FF00D0EF76E480EF66ED7EC01F00D0EF9
:103FB000DFEC01F00A0EDFEC01F001EEE1F012EEB1
:103FC00075F0410EE75204E0E6CFEEFFE82EFAD797
:103FD000EF6A416A01EEE1F0E86AEE5202E0E83E83
:103FE000FCD70401176F0101CC6B00010101CC511A
:103FF0000401175D0001D8A081EF20F0D8960101DF
:10400000D9A5D8860001D8B618EF20F00D0EF76EAE
:104010006C0EF66ED7EC01F0040E016E0401175120
:10402000CCEC00F00D0EDFEC01F00A0EDFEC01F03D
:104030000001D8960101D9A5D8860001D8B63EEF77
:1040400020F0690EDFEC01F03D0EDFEC01F0DFEC5B
:1040500001F0040E016E0101CC51CCEC00F00D0E0C
:10406000F76E7E0EF66ED7EC01F04150CCEC00F00E
:104070000D0EDFEC01F00A0EDFEC01F0000101EEA5
:10408000E1F00101CC51E926000EEA22EF500B6E5F
:10409000200E0B5C0001D8A454EF20F00101CC29C4
:1040A000416E000181EF20F0D8960101D9A5D88694
:1040B0000001D8B67BEF20F0690EDFEC01F03D0E79
:1040C000DFEC01F0DFEC01F0DFEC01F0040E016E3B
:1040D0000101CC51CCEC00F00D0EF76E8C0EF66E9B
:1040E000D7EC01F04150CCEC00F00D0EDFEC01F00C
:1040F0000A0EDFEC01F000010101CC2B0001D8A475
:1041000074D700EE43F011EEE1F04104E6CFEEFF8C
:10411000E82EFCD7EF6A00EE43F010EE43F0F5EC2A
:1041200002F000EE58F011EEE1F041500401175D8D
:10413000EAEC02F0EF6A41520001D8A4A3EF20F0AC
:1041400000EE58F0EE6A00EE58F010EE58F0F5EC84
:1041500002F001EE31F010EE58F0400EE75204E0AC
:10416000E6CFEEFFE82EFAD7EF6AD8960101D9A57F
:10417000D8860001D8B6CEEF20F00D0EF76E9C0E5B
:10418000F66ED7EC01F0040E016E4150CCEC00F05D
:104190000D0EDFEC01F00A0EDFEC01F0D896010104
:1041A000D9A5D8860001D8B6E9EF20F00D0EF76E3C
:1041B000AA0EF66ED7EC01F000EE43F0EE5003E0ED
:1041C000DFEC01F0FBD70D0EDFEC01F00A0EDFECA7
:1041D00001F0D8960101D9A5D8860001D8B604EF20
:1041E00021F00D0EF76EB80EF66ED7EC01F000EE72
:1041F00058F0EE5003E0DFEC01F0FBD70D0EDFECE2
:1042000001F00A0EDFEC01F00D0EF76EC60EF66E31
:1042100000EE43F001EC03F0D8A413EF21F0BFEC63
:104220003EF0F8EF25F00D0EF76ED00EF66E00EEB4
:1042300043F001EC03F0D8A422EF21F0E5EC3EF0CE
:10424000F8EF25F00D0EF76EDA0EF66E00EE43F085
:1042500001EC03F0D8A431EF21F00BEC3FF0F8EFC4
:1042600025F00D0EF76EE40EF66E00EE43F001EC55
:1042700003F0D8A440EF21F031EC3FF0F8EF25F047
:104280000D0EF76EEE0EF66E00EE43F001EC03F04D
:10429000D8A44FEF21F057EC3FF0F8EF25F00D0ECA
:1042A000F76EF80EF66E00EE43F001EC03F0D8A4C2
:1042B0005EEF21F07DEC3FF0F8EF25F00E0EF76E8B
:1042C000020EF66E00EE43F001EC03F0D8A46DEFA1
:1042D00021F0A3EC3FF0F8EF25F00E0EF76E0C0E78
:1042E000F66E00EE43F001EC03F0D8A47CEF21F071
:1042F000C9EC3FF0F8EF25F00E0EF76E160EF66ED5
:1043000000EE43F001EC03F0D8A48BEF21F0EFECCA
:104310003FF0F8EF25F00E0EF76E200EF66E00EE71
:1043200043F001EC03F0D8A49AEF21F015EC40F033
:10433000F8EF25F00E0EF76E2A0EF66E00EE43F043
:1043400001EC03F0D8A4A9EF21F03BEC40F0F8EF2A
:1043500025F00E0EF76E320EF66E00EE43F001EC15
:1043600003F0D8A4B8EF21F0A1EC40F0F8EF25F06D
:104370000E0EF76E3A0EF66E00EE43F001EC03F00F
:10438000D8A4D3EF21F00601098904EEA4F00E0EA3
:10439000F76E440EF66ED9EC02F0EF6A000128ECDD
:1043A0001EF0F8EF25F00E0EF76E5A0EF66E00EEC8
:1043B00043F001EC03F0D8A4EEEF21F006010999D7
:1043C00004EEA4F00E0EF76E640EF66ED9EC02F059
:1043D000EF6A000128EC1EF0F8EF25F00E0EF76EE4
:1043E0007A0EF66E00EE43F001EC03F0D8A409EF6C
:1043F00022F00601098B04EEA4F00E0EF76E840E77
:10440000F66ED9EC02F0EF6A000128EC1EF0F8EF2E
:1044100025F00E0EF76E9A0EF66E00EE43F001ECEC
:1044200003F0D8A424EF22F00601099B04EEA4F0C7
:104430000E0EF76EA60EF66ED9EC02F0EF6A0001D2
:1044400028EC1EF0F8EF25F00E0EF76EBE0EF66E9D
:1044500000EE43F001EC03F0D8A433EF22F007ECB8
:1044600041F0F8EF25F00E0EF76EC40EF66E00EE7A
:1044700043F001EC03F0D8A442EF22F03CEC41F011
:10448000F8EF25F00E0EF76ECA0EF66E00EE43F052
:1044900001EC03F0D8A451EF22F071EC41F0F8EFF9
:1044A00025F00E0EF76ED00EF66E00EE43F001EC26
:1044B00003F0D8A460EF22F0A6EC41F0F8EF25F06D
:1044C0000E0EF76ED60EF66E00EE43F001EC03F022
:1044D000D8A46FEF22F0DBEC41F0F8EF25F00E0EE0
:1044E000F76EDC0EF66E00EE43F001EC03F0D8A49C
:1044F0007EEF22F013EC42F0F8EF25F00E0EF76E8F
:10450000E00EF66E00EE43F001EC03F0D8A48DEF60
:1045100022F013EC42F0F8EF25F00E0EF76EE40EE9
:10452000F66E00EE43F001EC03F0D8A49CEF22F00D
:1045300059EC42F0F8EF25F00E0EF76EE80EF66E2D
:1045400000EE43F001EC03F0D8A4ABEF22F0E5EC71
:1045500042F0F8EF25F00E0EF76EEE0EF66E00EE5E
:1045600043F001EC03F0D8A4BAEF22F026EC2BF0D4
:10457000F8EF25F00E0EF76EF20EF66E00EE43F039
:1045800001EC03F0D8A4C9EF22F035EC2BF0F8EFE2
:1045900025F00E0EF76EF80EF66E00EE43F001EC0D
:1045A00003F0D8A4D8EF22F05FEC2BF0F8EF25F061
:1045B0000E0EF76EFC0EF66E00EE43F001EC03F00B
:1045C000D8A4E7EF22F047EC37F0F8EF25F00F0E14
:1045D000F76E000EF66E00EE43F001EC03F0D8A487
:1045E000F6EF22F0F3EC37F0F8EF25F00F0EF76E50
:1045F000080EF66E00EE43F001EC03F0D8A405EFD0
:1046000023F0C2EC31F0F8EF25F00F0EF76E100E2C
:10461000F66E00EE43F001EC03F0D8A414EF23F0A3
:10462000FDEC31F0F8EF25F00F0EF76E180EF66E78
:1046300000EE43F001EC03F0D8A423EF23F038ECB4
:1046400032F0F8EF25F00F0EF76E200EF66E00EE4A
:1046500043F001EC03F0D8A432EF23F073EC32F016
:10466000F8EF25F00F0EF76E280EF66E00EE43F011
:1046700001EC03F0D8A441EF23F0AEEC32F0F8EFF8
:1046800025F00F0EF76E300EF66E00EE43F001ECE3
:1046900003F0D8A450EF23F0E9EC32F0F8EF25F066
:1046A0000F0EF76E380EF66E00EE43F001EC03F0DD
:1046B000D8A45FEF23F024EC33F0F8EF25F00F0ED1
:1046C000F76E400EF66E00EE43F001EC03F0D8A456
:1046D0006EEF23F05FEC33F0F8EF25F00F0EF76E7E
:1046E000480EF66E00EE43F001EC03F0D8A47DEF27
:1046F00023F08DEC31F0F8EF25F00F0EF76E500E31
:10470000F66E00EE43F001EC03F0D8A48CEF23F03A
:104710009AEC33F0F8EF25F00F0EF76E580EF66EA8
:1047200000EE43F001EC03F0D8A49BEF23F0EFEC94
:1047300033F0F8EF25F00F0EF76E600EF66E00EE18
:1047400043F001EC03F0D8A4AAEF23F044EC34F0DA
:10475000F8EF25F00F0EF76E680EF66E00EE43F0E0
:1047600001EC03F0D8A4B9EF23F099EC34F0F8EFA2
:1047700025F00F0EF76E700EF66E00EE43F001ECB2
:1047800003F0D8A4C8EF23F050EC3EF0F8EF25F08A
:104790000F0EF76E780EF66E00EE43F001EC03F0AC
:1047A000D8A4D7EF23F06EEC3EF0F8EF25F00F0E13
:1047B000F76E820EF66E00EE43F001EC03F0D8A423
:1047C000E6EF23F0ACEC2AF0F8EF25F00F0EF76ED1
:1047D000860EF66E00EE43F001EC03F0D8A4F5EF80
:1047E00023F0A4EC2AF0F8EF25F00F0EF76E8C0EF4
:1047F000F66E00EE43F001EC03F0D8A404EF24F0D1
:1048000009EC50F0F8EF25F00F0EF76E920EF66EF1
:1048100000EE43F001EC03F0D8A413EF24F0E3EC36
:1048200046F0F8EF25F00F0EF76E980EF66E00EEDC
:1048300043F001EC03F0D8A422EF24F0C4EC43F0E1
:10484000F8EF25F00F0EF76E9E0EF66E00EE43F0B9
:1048500001EC03F0D8A431EF24F0ADEC4AF0F8EF0E
:1048600025F00F0EF76EA60EF66E00EE43F001EC8B
:1048700003F0D8A440EF24F0B7EC26F0F8EF25F0D1
:104880000F0EF76EAC0EF66E00EE43F001EC03F087
:10489000D8A45BEF24F00101D98104EEA4F00F0E3F
:1048A000F76EB40EF66ED9EC02F0EF6A000128EC58
:1048B0001EF0F8EF25F00F0EF76EC20EF66E00EE4A
:1048C00043F001EC03F0D8A476EF24F00101D99174
:1048D00004EEA4F00F0EF76ECC0EF66ED9EC02F0DB
:1048E000EF6A000128EC1EF0F8EF25F00F0EF76ECE
:1048F000DC0EF66E00EE43F001EC03F0D8A491EF6D
:1049000024F00101D98304EEA4F00F0EF76EE60E39
:10491000F66ED9EC02F0EF6A000128EC1EF0F8EF19
:1049200025F0100EF76E040EF66E00EE43F001EC6B
:1049300003F0D8A4ACEF24F00101D99304EEA4F065
:10494000100EF76E100EF66ED9EC02F0EF6A000151
:1049500028EC1EF0F8EF25F0100EF76E2E0EF66E16
:1049600000EE43F001EC03F0D8A4C7EF24F00101FE
:10497000D98504EEA4F0100EF76E3A0EF66ED9EC5F
:1049800002F0EF6A000128EC1EF0F8EF25F0100E9F
:10499000F76E500EF66E00EE43F001EC03F0D8A473
:1049A000E2EF24F00101D99504EEA4F0100EF76EA9
:1049B0005C0EF66ED9EC02F0EF6A000128EC1EF0F6
:1049C000F8EF25F0100EF76E740EF66E00EE43F061
:1049D00001EC03F0D8A4F1EF24F0FFEC25F0F8EFA0
:1049E00025F0100EF76E7A0EF66E00EE43F001EC35
:1049F00003F0D8A400EF25F032EC26F0F8EF25F014
:104A0000100EF76E840EF66E00EE43F001EC03F02C
:104A1000D8A40FEF25F02AEC2AF0F8EF25F0100EBD
:104A2000F76E8E0EF66E00EE43F001EC03F0D8A4A4
:104A30001EEF25F0D2EC2AF0F8EF25F0100EF76EFD
:104A4000980EF66E00EE43F001EC03F0D8A42DEFC3
:104A500025F0D2EC2AF0F8EF25F0100EF76E9C0E40
:104A6000F66E00EE43F001EC03F0D8A448EF25F019
:104A70000401A36B04EEA4F0100EF76EA60EF66E02
:104A8000D9EC02F0EF6A000128EC1EF0F8EF25F0F7
:104A9000100EF76EC20EF66E00EE43F001EC03F05E
:104AA000D8A464EF25F0010E0401A36F04EEA4F076
:104AB000100EF76ECA0EF66ED9EC02F0EF6A000126
:104AC00028EC1EF0F8EF25F0100EF76EF40EF66EDF
:104AD00000EE43F001EC03F0D8A473EF25F064EC92
:104AE0001CF0F8EF25F0100EF76EFA0EF66E00EEE1
:104AF00043F001EC03F0D8A482EF25F0B4EC2AF0E7
:104B0000F8EF25F0110EF76E080EF66E00EE43F08A
:104B100001EC03F0D8A491EF25F025EC43F0F8EF79
:104B200025F0110EF76E0E0EF66E00EE43F001EC5E
:104B300003F0D8A4A0EF25F089EF15F0F8EF25F0E9
:104B4000110EF76E160EF66E00EE43F001EC03F058
:104B5000D8A4AFEF25F08CEC3EF0F8EF25F0110E65
:104B6000F76E1E0EF66E00EE43F001EC03F0D8A4D3
:104B7000BEEF25F0A1EC3EF0F8EF25F0110EF76E38
:104B8000260EF66E00EE43F001EC03F0D8A4CDEF54
:104B900025F0CBEC30F0F8EF25F0110EF76E2A0E71
:104BA000F66E00EE43F001EC03F0D8A4DCEF25F044
:104BB000D9EC3DF0F8EF25F0110EF76E320EF66EDF
:104BC00000EE43F001EC03F0D8A4EBEF25F0FDEC90
:104BD0003DF0F8EF25F0110EF76E380EF66E00EE90
:104BE00043F001EC03F0D8A4F8EF25F0B0EC3DF071
:104BF0000401A26BA16B00012DEC18F0120002EE73
:104C0000CAF0110EF76E3E0EF66ED9EC02F011EE00
:104C1000DCF0040EE75204E0E6CFEEFFE82EFAD710
:104C2000110EF76E460EF66ED9EC02F015EEDCF0C2
:104C3000060EE75204E0E6CFEEFFE82EFAD7110E9B
:104C4000F76E500EF66ED9EC02F0020E016E050101
:104C5000E551CCEC00F0EF6A000175EC1CF01DECA6
:104C60001FF012000501E5510A0DF3CF1CF0F4CF3F
:104C70001DF026EC02F00001C2DF12000401A35374
:104C80000001D8A478EF26F002EECAF0110EF76EFC
:104C90005C0EF66ED9EC02F0020E016EE86A82B884
:104CA000010ECCEC00F0020E016EE86A82BA010E31
:104CB000CCEC00F0020E016EE86A81B0010ECCEC83
:104CC00000F0020E016EE86A81B2010ECCEC00F039
:104CD000020E016EE86A81B4010ECCEC00F0300ED9
:104CE000EE6EEE6EEE6EEF6A75EC1CF01DEC1FF0D2
:104CF000010E0401A35D0001D8A4B3EF26F002EE7B
:104D0000CAF0110EF76E640EF66ED9EC02F0020EC8
:104D1000016EE86A82B8010ECCEC00F0020E016E62
:104D2000E86A82BA010ECCEC00F0020E016EE86A6D
:104D300081B0010ECCEC00F0020E016EE86A81B287
:104D4000010ECCEC00F0020E016EE86A81B4010E97
:104D5000CCEC00F0300EEE6EEE6EEE6EEF6A75EC9F
:104D60001CF01DEC1FF0140E24EC02F012000401E4
:104D7000A3530001D8A445EF28F002EECAF0110EAB
:104D8000F76E6C0EF66ED9EC02F0020E016EE86A58
:104D900082B8010ECCEC00F0020E016EE86A82BA15
:104DA000010ECCEC00F0020E016EE86A81B0010E3B
:104DB000CCEC00F0020E016EE86A81B2010ECCEC80
:104DC00000F0020E016EE86A81B4010ECCEC00F036
:104DD000300EEE6EEE6EEE6EEF6A75EC1CF01DECB2
:104DE0001FF0140E24EC02F002EECAF0110EF76E62
:104DF000740EF66ED9EC02F0020E016E3AC52FF079
:104E000039C52EF038C52DF037C52CF0030EFEEC59
:104E100000F02C0EEE6E020E016E3EC52FF03DC569
:104E20002EF03CC52DF03BC52CF0030EFEEC00F03F
:104E30002C0EEE6E020E016E42C52FF041C52EF013
:104E400040C52DF03FC52CF0030EFEEC00F02C0EFB
:104E5000EE6E020E016E46C52FF045C52EF044C51C
:104E60002DF043C52CF0030EFEEC00F0EF6A75EC5C
:104E70001CF01DEC1FF0140E24EC02F002EECAF040
:104E8000110EF76E7C0EF66ED9EC02F0020E016E7A
:104E9000086AEEC521F0EDC520F0CFEC00F02C0E35
:104EA000EE6E020E016E086AF0C521F0EFC520F02B
:104EB000CFEC00F02C0EEE6E020E016E086AF2C509
:104EC00021F0F1C520F0CFEC00F02C0EEE6E020EBA
:104ED000016E086AF4C521F0F3C520F0CFEC00F0B4
:104EE0002C0EEE6E020E016E086AF6C521F0F5C5B5
:104EF00020F0CFEC00F02C0EEE6E020E016E086A70
:104F0000F8C521F0F7C520F0CFEC00F02C0EEE6EC6
:104F1000020E016E086AFAC521F0F9C520F0CFEC47
:104F200000F02C0EEE6E020E016E000ECCEC00F0C6
:104F30002C0EEE6E020E016EE86A060109B9010E32
:104F4000CCEC00F0EF6A000175EC1CF01DEC1FF0DA
:104F5000140E24EC02F002EECAF0110EF76E840E6D
:104F6000F66ED9EC02F0020E016E086AFCC521F063
:104F7000FBC520F0CFEC00F02C0EEE6E020E016EA1
:104F8000086AFEC521F0FDC520F0CFEC00F02C0E24
:104F9000EE6E020E016E086A00C621F0FFC520F019
:104FA000CFEC00F02C0EEE6E020E016E086A02C607
:104FB00021F001C620F0CFEC00F02C0EEE6E020EB8
:104FC000016E086A04C621F003C620F0CFEC00F0A1
:104FD0002C0EEE6E020E016E086A06C621F005C6A2
:104FE00020F0CFEC00F02C0EEE6E020E016E086A7F
:104FF00008C621F007C620F0CFEC00F02C0EEE6EB4
:10500000020E016E000ECCEC00F02C0EEE6E020EC5
:10501000016EE86A060109BB010ECCEC00F0EF6AF4
:10502000000175EC1CF01DEC1FF0140E24EC02F0D6
:1050300002EECAF0110EF76E8C0EF66ED9EC02F08D
:10504000020E016E0501E551CCEC00F02C0EEE6E67
:10505000020E016E086AD9C521F0D8C520F0CFEC48
:1050600000F02C0EEE6E020E016E086ADBC521F018
:10507000DAC520F0CFEC00F0EF6A000175EC1CF00F
:105080001DEC1FF0140E24EC02F0010E0401A35DD0
:105090000001D8A4D4EF29F002EECAF0110EF76E89
:1050A000940EF66ED9EC02F0020E016EE86A82B838
:1050B000010ECCEC00F0020E016EE86A82BA010E1D
:1050C000CCEC00F0020E016EE86A81B0010ECCEC6F
:1050D00000F0020E016EE86A81B2010ECCEC00F025
:1050E000020E016EE86A81B4010ECCEC00F0300EC5
:1050F000EE6EEE6EEE6EEF6A75EC1CF01DEC1FF0BE
:10510000140E24EC02F002EECAF0110EF76E9C0EA3
:10511000F66ED9EC02F0020E016E3AC52FF039C5D9
:105120002EF038C52DF037C52CF0030EFEEC00F044
:105130002C0EEE6E020E016E3EC52FF03DC52EF018
:105140003CC52DF03BC52CF0030EFEEC00F02C0E00
:10515000EE6E020E016E42C52FF041C52EF040C525
:105160002DF03FC52CF0030EFEEC00F02C0EEE6E81
:10517000020E016E46C52FF045C52EF044C52DF038
:1051800043C52CF0030EFEEC00F0EF6A75EC1CF04A
:105190001DEC1FF0140E24EC02F002EECAF0110E0A
:1051A000F76EA40EF66ED9EC02F0020E016E086ADC
:1051B000EEC521F0EDC520F0CFEC00F02C0EEE6E28
:1051C000020E016E086AF0C521F0EFC520F0CFECA9
:1051D00000F02C0EEE6E020E016E086AF2C521F090
:1051E000F1C520F0CFEC00F02C0EEE6E020E016E39
:1051F000086AF4C521F0F3C520F0CFEC00F02C0EC6
:10520000EE6E020E016E086AF6C521F0F5C520F0BB
:10521000CFEC00F02C0EEE6E020E016E086AF8C59F
:1052200021F0F7C520F0CFEC00F02C0EEE6E020E50
:10523000016E086AFAC521F0F9C520F0CFEC00F044
:105240002C0EEE6E020E016E000ECCEC00F02C0E59
:10525000EE6E020E016EE86A060109B9010ECCEC91
:1052600000F0EF6A000175EC1CF01DEC1FF0140E4D
:1052700024EC02F002EECAF0110EF76EAC0EF66EE0
:10528000D9EC02F0020E016E086AFCC521F0FBC5E4
:1052900020F0CFEC00F02C0EEE6E020E016E086ACC
:1052A000FEC521F0FDC520F0CFEC00F02C0EEE6E17
:1052B000020E016E086A00C621F0FFC520F0CFEC97
:1052C00000F02C0EEE6E020E016E086A02C621F08E
:1052D00001C620F0CFEC00F02C0EEE6E020E016E37
:1052E000086A04C621F003C620F0CFEC00F02C0EB3
:1052F000EE6E020E016E086A06C621F005C620F0A9
:10530000CFEC00F02C0EEE6E020E016E086A08C69D
:1053100021F007C620F0CFEC00F02C0EEE6E020E4E
:10532000016E000ECCEC00F02C0EEE6E020E016E43
:10533000E86A060109BB010ECCEC00F0EF6A00013F
:1053400075EC1CF01DEC1FF0140E24EC02F002EEC4
:10535000CAF0110EF76EB40EF66ED9EC02F0020E22
:10536000016E0501E551CCEC00F02C0EEE6E020E44
:10537000016E086AD9C521F0D8C520F0CFEC00F045
:105380002C0EEE6E020E016E086ADBC521F0DAC546
:1053900020F0CFEC00F0EF6A000175EC1CF01DEC82
:1053A0001FF0140E24EC02F01200110EF76EBC0E6A
:1053B000F66E01EEDCF001EC03F0D8A4FCEF29F06E
:1053C000010E0101CC6F0001040E0101CC5D000152
:1053D000D8B0FAEF29F094928292FA0E24EC02F0FF
:1053E00094928282FA0E24EC02F00101CC2B00018F
:1053F000D8A4E9D729EF2AF0010E0101CC6F0001F2
:10540000030E0101CC5D0001D8B029EF2AF094927F
:105410008292010E1D6EF40E25EC02F094928282AF
:10542000C80E24EC02F094928292010E1D6EF40ECE
:1054300025EC02F094928282C80E24EC02F0010E58
:105440001D6E900E25EC02F00101CC2B0001D8A4BA
:10545000D6D7120001EEDCF0460EEE6E410EEE6E77
:10546000490EEE6E4C0EEE6EEF6A12009DEC2AF0C5
:1054700001EE31F0110EF76EC00EF66ED9EC02F0AF
:10548000020E016E0501E551CCEC00F0110EF76E35
:10549000D40EF66ED9EC02F0EF6A000164EC1CF059
:1054A000010E0101CC6F0001040E0101CC5D000171
:1054B000D8B080EF2AF094928292820E026E040E8F
:1054C000096E010E046EF40E036E030E216EE80EDB
:1054D000206E33EC00F094928282820E026E040EF3
:1054E000096E010E046EF40E036E010E216E900E15
:1054F000206E33EC00F00101CC2B0001D8A4D3D7EF
:1055000005EE92F0460EEE6E410EEE6E490EEE6E18
:105510004C0EEE6EEF6A81EC2BF094928292010EAB
:105520001D6EF40E25EC02F094928282010E1D6E27
:10553000F40E25EC02F0F1D712008298829A819045
:1055400081928194120012000501256B01016B6BA1
:105550000601099700011200010E0501256F010ED9
:1055600001016B6F0001120001EE31F084EC00F0DC
:105570000501EB6F21C0ECF504EEA4F0110EF76EFF
:10558000E60EF66ED9EC02F0020E016E086AECC56A
:1055900021F0EBC520F0CFEC00F0EF6A000128EC21
:1055A0001EF01200CADF2D0E0101CC6F010ED46F68
:1055B0000001090E0101D45D0001D8B024EF2BF0E9
:1055C000949882880101CC5124EC02F0949882983E
:1055D000949A828ACC5124EC02F0949A829A939005
:1055E0008180CC5124EC02F093908190939281823F
:1055F000CC5124EC02F09392819293948184CC510B
:1056000024EC02F09394819493928182CC5124EC07
:1056100002F09392819293908180CC5124EC02F01D
:1056200093908190949A828ACC5124EC02F0949ABF
:10563000829A94988288CC5124EC02F094988298B3
:10564000D42B0001D8A4B4D778DF120005EE92F075
:1056500011EE31F0360EE75204E0E6CFEEFFE82E11
:10566000FAD7EF6A81EC2BF01200120EF76E000EE3
:10567000F66E01EE31F001EC03F0D8A450EF2BF000
:1056800005012A8504EEA4F0120EF76E040EF66EE4
:10569000D9EC02F0EF6A000128EC1EF05EEF2BF06F
:1056A00005012A9504EEA4F0120EF76E120EF66EA6
:1056B000D9EC02F0EF6A000128EC1EF0120001EEB6
:1056C00031F084EC00F00501906F040E196EB00EFD
:1056D000186E1D6A90C51CF09CEC02F08E6F19C00C
:1056E0008FF504EEA4F0120EF76E220EF66ED9ECD2
:1056F00002F0020E016E9051CCEC00F0EF6A000156
:10570000120004EEA4F0120EF76E340EF66ED9EC11
:1057100002F015EE92F0320EE75204E0E6CFEEFF13
:10572000E82EFAD7EF6A28EC1EF0040E196EB00EC0
:10573000186E1D6A90C51CF09CEC02F005018E6F7E
:1057400019C08FF59492828205EE92F0E86AEE52CB
:1057500002E0E83EFCD7916F010E0101CC6F000121
:105760000101CC510501915D0001D8A07BEF2EF025
:1057700005EEC5F015EE92F0CCC1F3FF010EE1ECA1
:1057800002F0EF6A410E0501C55D0001D8A4D2EF19
:105790002BF005EECAF02E0EEE6E2D0EEE6EEF6AB9
:1057A00073EF2EF0420E0501C55D0001D8A4E4EFB1
:1057B0002BF005EECAF02D0EEE6E2E0EEE6EEE6E96
:1057C000EE6EEF6A73EF2EF0430E0501C55D00012A
:1057D000D8A4F8EF2BF005EECAF02D0EEE6E2E0ECB
:1057E000EE6E2D0EEE6E2E0EEE6EEF6A73EF2EF055
:1057F000440E0501C55D0001D8A409EF2CF005EEAB
:10580000CAF02D0EEE6E2E0EEE6EEE6EEF6A73EF98
:105810002EF0450E0501C55D0001D8A417EF2CF050
:1058200005EECAF02E0EEE6EEF6A73EF2EF0460E06
:105830000501C55D0001D8A42AEF2CF005EECAF0E1
:105840002E0EEE6EEE6E2D0EEE6E2E0EEE6EEF6ADC
:1058500073EF2EF0470E0501C55D0001D8A43BEFA4
:105860002CF005EECAF02D0EEE6EEE6E2E0EEE6EE4
:10587000EF6A73EF2EF0480E0501C55D0001D8A454
:105880004CEF2CF005EECAF02E0EEE6EEE6EEE6EC4
:10589000EE6EEF6A73EF2EF0490E0501C55D000153
:1058A000D8A45BEF2CF005EECAF02E0EEE6EEE6E75
:1058B000EF6A73EF2EF04A0E0501C55D0001D8A412
:1058C0006DEF2CF005EECAF02E0EEE6E2D0EEE6E84
:1058D000EE6EEE6EEF6A73EF2EF04B0E0501C55DB6
:1058E0000001D8A47FEF2CF005EECAF02D0EEE6E6D
:1058F0002E0EEE6E2D0EEE6EEF6A73EF2EF04C0E46
:105900000501C55D0001D8A492EF2CF005EECAF0A8
:105910002E0EEE6E2D0EEE6E2E0EEE6EEE6EEF6A0B
:1059200073EF2EF04D0E0501C55D0001D8A4A1EF67
:105930002CF005EECAF02D0EEE6EEE6EEF6A73EFF0
:105940002EF04E0E0501C55D0001D8A4B1EF2CF07C
:1059500005EECAF02D0EEE6E2E0EEE6EEF6A73EFB0
:105960002EF04F0E0501C55D0001D8A4C1EF2CF04B
:1059700005EECAF02D0EEE6EEE6EEE6EEF6A73EF70
:105980002EF0500E0501C55D0001D8A4D4EF2CF017
:1059900005EECAF02E0EEE6E2D0EEE6EEE6E2E0E93
:1059A000EE6EEF6A73EF2EF0510E0501C55D00013A
:1059B000D8A4E7EF2CF005EECAF02D0EEE6EEE6ED9
:1059C0002E0EEE6E2D0EEE6EEF6A73EF2EF0520E6F
:1059D0000501C55D0001D8A4F9EF2CF005EECAF071
:1059E0002E0EEE6E2D0EEE6E2E0EEE6EEF6A73EF35
:1059F0002EF0530E0501C55D0001D8A409EF2DF06E
:105A000005EECAF02E0EEE6EEE6EEE6EEF6A73EFDE
:105A10002EF0540E0501C55D0001D8A417EF2DF03E
:105A200005EECAF02D0EEE6EEF6A73EF2EF0550EF6
:105A30000501C55D0001D8A428EF2DF005EECAF0E0
:105A40002E0EEE6EEE6E2D0EEE6EEF6A73EF2EF0F2
:105A5000560E0501C55D0001D8A43AEF2DF005EE04
:105A6000CAF02E0EEE6EEE6EEE6E2D0EEE6EEF6A3C
:105A700073EF2EF0570E0501C55D0001D8A44BEF62
:105A80002DF005EECAF02E0EEE6E2D0EEE6EEE6EC1
:105A9000EF6A73EF2EF0580E0501C55D0001D8A422
:105AA0005EEF2DF005EECAF02D0EEE6E2E0EEE6EB0
:105AB000EE6E2D0EEE6EEF6A73EF2EF0590E0501AD
:105AC000C55D0001D8A471EF2DF005EECAF02D0ED2
:105AD000EE6E2E0EEE6E2D0EEE6EEE6EEF6A73EF24
:105AE0002EF05A0E0501C55D0001D8A483EF2DF0FC
:105AF00005EECAF02D0EEE6EEE6E2E0EEE6EEE6E12
:105B0000EF6A73EF2EF0300E0501C55D0001D8A4D9
:105B100095EF2DF005EECAF02D0EEE6EEE6EEE6EE8
:105B2000EE6EEE6EEF6A73EF2EF0310E0501C55D7D
:105B30000001D8A4A8EF2DF005EECAF02E0EEE6EEF
:105B40002D0EEE6EEE6EEE6EEE6EEF6A73EF2EF0D1
:105B5000320E0501C55D0001D8A4BBEF2DF005EEA6
:105B6000CAF02E0EEE6EEE6E2D0EEE6EEE6EEE6E38
:105B7000EF6A73EF2EF0330E0501C55D0001D8A466
:105B8000CEEF2DF005EECAF02E0EEE6EEE6EEE6E3E
:105B90002D0EEE6EEE6EEF6A73EF2EF0340E0501F1
:105BA000C55D0001D8A4E0EF2DF005EECAF02E0E81
:105BB000EE6EEE6EEE6E2D0EEE6EEF6A73EF2EF061
:105BC000350E0501C55D0001D8A4F2EF2DF005EEFC
:105BD000CAF02E0EEE6EEE6EEE6EEE6EEE6EEF6AAA
:105BE00073EF2EF0360E0501C55D0001D8A405EF58
:105BF0002EF005EECAF02D0EEE6E2E0EEE6EEE6E4F
:105C0000EE6EEE6EEF6A73EF2EF0370E0501C55D96
:105C10000001D8A418EF2EF005EECAF02D0EEE6E9E
:105C2000EE6E2E0EEE6EEE6EEE6EEF6A73EF2EF0EF
:105C3000380E0501C55D0001D8A42BEF2EF005EE4E
:105C4000CAF02D0EEE6EEE6EEE6E2E0EEE6EEE6E57
:105C5000EF6A73EF2EF0390E0501C55D0001D8A47F
:105C60003EEF2EF005EECAF02D0EEE6EEE6EEE6EED
:105C7000EE6E2E0EEE6EEF6A73EF2EF02F0E050114
:105C8000C55D0001D8A453EF2EF005EECAF02D0E2D
:105C9000EE6E2E0EEE6EEE6E2D0EEE6E2E0EEE6E85
:105CA000EF6A73EF2EF03D0E0501C55D0001D8A42B
:105CB00067EF2EF005EECAF02D0EEE6E2E0EEE6E94
:105CC000EE6EEE6E2D0EEE6EEF6A73EF2EF0200E7E
:105CD0000501C55D0001D8A473EF2EF005EECAF0F2
:105CE000200EEE6EEF6A7CEC2EF00101CC2B000151
:105CF000D8A4AFEF2BF0120005EECAF0E86AEE521E
:105D000002E0E83EFCD70101D46F010ED76F00011D
:105D10000101D751D45D0001D8A01DEF2FF005EE91
:105D2000C7F015EECAF0D7C1F3FF010EE1EC02F0A7
:105D3000EF6A2E0E0501C75D0001D8A4C8EF2EF052
:105D400094928292D89605012AA5D8860001D8B6E9
:105D5000ACEF2EF093948184820E026E040E096ED5
:105D60008FC504F08EC503F08DC521F08CC520F0E1
:105D700033EC00F0D89605012AA5D8860001D8B6E4
:105D8000C4EF2EF0939481949492828212EF2FF0BC
:105D90002D0E0501C75D0001D8A4FDEF2EF09492F1
:105DA0008292D89605012AA5D8860001D8B6DBEFE5
:105DB0002EF093948184820E026E040E096E05010A
:105DC0008F51030DF3CF04F08E51030DF3CF03F089
:105DD000F45004268DC521F08CC520F033EC00F082
:105DE000D8962AA5D8860001D8B6F9EF2EF093945C
:105DF00081949492828212EF2FF0200E0501C75DEC
:105E00000001D8A411EF2FF005018F51030DF3CF3E
:105E10001DF08E51030DF3CF1CF0F4501D2626EC1F
:105E200002F000018FC51DF005018E5125EC02F036
:105E30000101D72B0001D8A46AD705018F51030DAA
:105E4000F3CF1DF08E51030DF3CF1CF0F4501D263F
:105E500026EC02F000011200000E0DEC02F005012C
:105E60002F6F2DC030F5176A166A156A8F0E146EE3
:105E700030C511F02FC510F0D0EC04F018EC04F090
:105E800013C0D2F112C0D1F111C0D0F110C0CFF1C6
:105E9000136A126A200E116E810E106ED2C117F0B5
:105EA000D1C116F0D0C115F0CFC114F080EC04F0D0
:105EB00013C02FF012C02EF011C02DF010C02CF026
:105EC0002FC013F02EC012F02DC011F02CC010F016
:105ED0002EC517F02DC516F02CC515F02BC514F0E6
:105EE00080EC04F013C03AF512C039F511C038F552
:105EF00010C037F53AC513F039C512F038C511F0A6
:105F000037C510F04AC517F049C516F048C515F059
:105F100047C514F07EEC03F013C03AF512C039F512
:105F200011C038F510C037F5010E0DEC02F0316FDD
:105F30002DC032F5176A166A156A8F0E146E32C5B7
:105F400011F031C510F0D0EC04F018EC04F013C0DF
:105F5000D2F112C0D1F111C0D0F110C0CFF1136A4B
:105F6000126A200E116E810E106ED2C117F0D1C1CF
:105F700016F0D0C115F0CFC114F080EC04F013C0BE
:105F80002FF012C02EF011C02DF010C02CF02FC039
:105F900013F02EC012F02DC011F02CC010F02EC541
:105FA00017F02DC516F02CC515F02BC514F080EC9C
:105FB00004F013C03EF512C03DF511C03CF510C011
:105FC0003BF53EC513F03DC512F03CC511F03BC595
:105FD00010F04EC517F04DC516F04CC515F04BC569
:105FE00014F07EEC03F013C03EF512C03DF511C075
:105FF0003CF510C03BF5020E0DEC02F0336F2DC0E6
:1060000034F5176A166A156A8F0E146E34C511F0CE
:1060100033C510F0D0EC04F018EC04F013C0D2F14A
:1060200012C0D1F111C0D0F110C0CFF1136A126AC1
:10603000200E116E810E106ED2C117F0D1C116F074
:10604000D0C115F0CFC114F080EC04F013C02FF0D4
:1060500012C02EF011C02DF010C02CF02FC013F084
:106060002EC012F02DC011F02CC010F02EC517F06C
:106070002DC516F02CC515F02BC514F080EC04F0DE
:1060800013C042F512C041F511C040F510C03FF5F4
:1060900042C513F041C512F040C511F03FC510F0E4
:1060A00052C517F051C516F050C515F04FC514F084
:1060B0007EEC03F013C042F512C041F511C040F56B
:1060C00010C03FF5030E0DEC02F0356F2DC036F514
:1060D000176A166A156A8F0E146E36C511F035C52B
:1060E00010F0D0EC04F018EC04F013C0D2F112C0A0
:1060F000D1F111C0D0F110C0CFF1136A126A200E95
:10610000116E810E106ED2C117F0D1C116F0D0C140
:1061100015F0CFC114F080EC04F013C02FF012C0C2
:106120002EF011C02DF010C02CF02FC013F02EC097
:1061300012F02DC011F02CC010F02EC517F02DC597
:1061400016F02CC515F02BC514F080EC04F013C02C
:1061500046F512C045F511C044F510C043F546C5DB
:1061600013F045C512F044C511F043C510F056C5F3
:1061700017F055C516F054C515F053C514F07EEC54
:1061800003F013C046F512C045F511C044F510C028
:1061900043F50001120004EEA4F0120EF76E3E0E5D
:1061A000F66ED9EC02F0EF6A28EC1EF00A0E24EC31
:1061B00002F052DE04EEA4F0120EF76E640EF66EDC
:1061C000D9EC02F0020E016E3AC52FF039C52EF05F
:1061D00038C52DF037C52CF0030EFEEC00F0120E82
:1061E000F76E740EF66ED9EC02F0020E016E086ABC
:1061F00030C521F02FC520F0CFEC00F0290EEE6E57
:10620000EF6A28EC1EF004EEA4F0120EF76E7E0E7C
:10621000F66ED9EC02F0020E016E3EC52FF03DC5C0
:106220002EF03CC52DF03BC52CF0030EFEEC00F02B
:10623000120EF76E8E0EF66ED9EC02F0020E016EA3
:10624000086A32C521F031C520F0CFEC00F0290EEC
:10625000EE6EEF6A28EC1EF004EEA4F0120EF76E5C
:10626000980EF66ED9EC02F0020E016E42C52FF0C8
:1062700041C52EF040C52DF03FC52CF0030EFEECBD
:1062800000F0120EF76EA80EF66ED9EC02F0020EB8
:10629000016E086A34C521F033C520F0CFEC00F060
:1062A000290EEE6EEF6A28EC1EF004EEA4F0120E3A
:1062B000F76EB20EF66ED9EC02F0020E016E46C514
:1062C0002FF045C52EF044C52DF043C52CF0030E2C
:1062D000FEEC00F0120EF76EC20EF66ED9EC02F074
:1062E000020E016E086A36C521F035C520F0CFECEC
:1062F00000F0290EEE6EEF6A28EC1EF004EEA4F01A
:10630000120EF76ECC0EF66ED9EC02F0EF6A28ECA6
:106310001EF00A0E24EC02F01200120EF76EF20EBE
:10632000F66E01EE31F001EC03F0D8A4A7EF31F0E6
:10633000010E01016C6F04EEA4F0120EF76EF60E62
:10634000F66ED9EC02F0EF6A000128EC1EF0130E95
:10635000F76E120EF66E01EE31F001EC03F0D8A4E8
:10636000C0EF31F001016C6B04EEA4F0130EF76E78
:10637000160EF66ED9EC02F0EF6A000128EC1EF062
:106380001200120001EE31F084EC00F020C010F099
:1063900021C011F022C012F023C013F0D2EC04F09F
:1063A00013C05AF512C059F511C058F510C057F571
:1063B00001EEA0F0020E016E5AC52FF059C52EF065
:1063C00058C52DF057C52CF0030EFEEC00F0EF6A17
:1063D00004EEA4F0130EF76E320EF66ED9EC02F056
:1063E00011EEA0F0140EE75204E0E6CFEEFFE82E27
:1063F000FAD7EF6A28EC1EF0120001EE31F084ECBF
:1064000000F020C010F021C011F022C012F023C013
:1064100013F0D2EC04F013C05EF512C05DF511C0AC
:106420005CF510C05BF501EEA0F0020E016E5EC5DA
:106430002FF05DC52EF05CC52DF05BC52CF0030E72
:10644000FEEC00F0EF6A04EEA4F0130EF76E480EB7
:10645000F66ED9EC02F011EEA0F0140EE75204E053
:10646000E6CFEEFFE82EFAD7EF6A28EC1EF0120016
:1064700001EE31F084EC00F020C010F021C011F0EA
:1064800022C012F023C013F0D2EC04F013C062F566
:1064900012C061F511C060F510C05FF501EEA0F00B
:1064A000020E016E62C52FF061C52EF060C52DF0A1
:1064B0005FC52CF0030EFEEC00F0EF6A04EEA4F0D2
:1064C000130EF76E5E0EF66ED9EC02F011EEA0F030
:1064D000140EE75204E0E6CFEEFFE82EFAD7EF6A9B
:1064E00028EC1EF0120001EE31F084EC00F020C028
:1064F00010F021C011F022C012F023C013F0D2EC32
:1065000004F013C066F512C065F511C064F510C043
:1065100063F501EEA0F0020E016E66C52FF065C5B1
:106520002EF064C52DF063C52CF0030EFEEC00F0D8
:10653000EF6A04EEA4F0130EF76E740EF66ED9EC4B
:1065400002F011EEA0F0140EE75204E0E6CFEEFFE9
:10655000E82EFAD7EF6A28EC1EF0120001EE31F0B7
:1065600084EC00F020C010F021C011F022C012F025
:1065700023C013F0D2EC04F013C06AF512C069F521
:1065800011C068F510C067F501EEA0F0020E016EB3
:106590006AC52FF069C52EF068C52DF067C52CF0CF
:1065A000030EFEEC00F0EF6A04EEA4F0130EF76E9B
:1065B0008A0EF66ED9EC02F011EEA0F0140EE7523E
:1065C00004E0E6CFEEFFE82EFAD7EF6A28EC1EF0E3
:1065D000120001EE31F084EC00F020C010F021C078
:1065E00011F022C012F023C013F0D2EC04F013C05B
:1065F0006EF512C06DF511C06CF510C06BF501EEB3
:10660000A0F0020E016E6EC52FF06DC52EF06CC5A8
:106610002DF06BC52CF0030EFEEC00F0EF6A04EEDB
:10662000A4F0130EF76EA00EF66ED9EC02F011EE88
:10663000A0F0140EE75204E0E6CFEEFFE82EFAD702
:10664000EF6A28EC1EF0120001EE31F084EC00F04D
:1066500020C010F021C011F022C012F023C013F0AE
:10666000D2EC04F013C072F512C071F511C070F5D0
:1066700010C06FF501EEA0F0020E016E72C52FF092
:1066800071C52EF070C52DF06FC52CF0030EFEEC19
:1066900000F0EF6A04EEA4F0130EF76EB60EF66E7D
:1066A000D9EC02F011EEA0F0140EE75204E0E6CFB0
:1066B000EEFFE82EFAD7EF6A28EC1EF0120001EE8A
:1066C00031F084EC00F020C010F021C011F022C0A5
:1066D00012F023C013F0D2EC04F013C076F512C010
:1066E00075F511C074F510C073F501EEA0F0020E3F
:1066F000016E76C52FF075C52EF074C52DF073C5EB
:106700002CF0030EFEEC00F0EF6A04EEA4F0130E82
:10671000F76ECC0EF66ED9EC02F011EEA0F0140E6E
:10672000E75204E0E6CFEEFFE82EFAD7EF6A28EC56
:106730001EF0120001EE31F084EC00F020C010F0E9
:1067400021C011F022C012F023C013F0D2EC04F0EB
:1067500013C0D2F112C0D1F111C0D0F110C0CFF1ED
:106760006F0E136E120E126E030E116E750E106EFA
:10677000D2C117F0D1C116F0D0C115F0CFC114F0BD
:1067800080EC04F013C04AF512C049F511C048F579
:1067900010C047F501EEA0F0020E016E4AC52FF0C1
:1067A00049C52EF048C52DF047C52CF0030EFEEC70
:1067B00000F0EF6A04EEA4F0130EF76EE20EF66E30
:1067C000D9EC02F011EEA0F0140EE75204E0E6CF8F
:1067D000EEFFE82EFAD7EF6A28EC1EF0120001EE69
:1067E00031F084EC00F020C010F021C011F022C084
:1067F00012F023C013F0D2EC04F013C0D2F112C097
:10680000D1F111C0D0F110C0CFF16F0E136E120E86
:10681000126E030E116E750E106ED2C117F0D1C13B
:1068200016F0D0C115F0CFC114F080EC04F013C005
:106830004EF512C04DF511C04CF510C04BF501EEF0
:10684000A0F0020E016E4EC52FF04DC52EF04CC5C6
:106850002DF04BC52CF0030EFEEC00F0EF6A04EEB9
:10686000A4F0140EF76E080EF66ED9EC02F011EEDD
:10687000A0F0140EE75204E0E6CFEEFFE82EFAD7C0
:10688000EF6A28EC1EF0120001EE31F084EC00F00B
:1068900020C010F021C011F022C012F023C013F06C
:1068A000D2EC04F013C0D2F112C0D1F111C0D0F17A
:1068B00010C0CFF16F0E136E120E126E030E116E1A
:1068C000750E106ED2C117F0D1C116F0D0C115F0FF
:1068D000CFC114F080EC04F013C052F512C051F592
:1068E00011C050F510C04FF501EEA0F0020E016E80
:1068F00052C52FF051C52EF050C52DF04FC52CF0CC
:10690000030EFEEC00F0EF6A04EEA4F0140EF76E36
:106910002E0EF66ED9EC02F011EEA0F0140EE75236
:1069200004E0E6CFEEFFE82EFAD7EF6A28EC1EF07F
:10693000120001EE31F084EC00F020C010F021C014
:1069400011F022C012F023C013F0D2EC04F013C0F7
:10695000D2F112C0D1F111C0D0F110C0CFF16F0E41
:10696000136E120E126E030E116E750E106ED2C1E2
:1069700017F0D1C116F0D0C115F0CFC114F080ECE2
:1069800004F013C056F512C055F511C054F510C0EF
:1069900053F501EEA0F0020E016E56C52FF055C55D
:1069A0002EF054C52DF053C52CF0030EFEEC00F074
:1069B000EF6A04EEA4F0140EF76E540EF66ED9ECE6
:1069C00002F011EEA0F0140EE75204E0E6CFEEFF65
:1069D000E82EFAD7EF6A28EC1EF012003AC513F041
:1069E00039C512F038C511F037C510F05AC517F087
:1069F00059C516F058C515F057C514F00AEC03F048
:106A00000108D8B41EEF35F0AFEC35F06AC513F0CD
:106A100069C512F068C511F067C510F03AC517F0E6
:106A200039C516F038C515F037C514F00AEC03F077
:106A30000108D8B41EEF35F07BEC36F03EC513F0FC
:106A40003DC512F03CC511F03BC510F05EC517F016
:106A50005DC516F05CC515F05BC514F00AEC03F0DB
:106A60000108D8B44EEF35F0E2EC35F06EC513F006
:106A70006DC512F06CC511F06BC510F03EC517F076
:106A80003DC516F03CC515F03BC514F00AEC03F00B
:106A90000108D8B44EEF35F0AEEC36F042C513F035
:106AA00041C512F040C511F03FC510F062C517F0A6
:106AB00061C516F060C515F05FC514F00AEC03F06F
:106AC0000108D8B47EEF35F015EC36F072C513F03E
:106AD00071C512F070C511F06FC510F042C517F006
:106AE00041C516F040C515F03FC514F00AEC03F09F
:106AF0000108D8B47EEF35F0E1EC36F046C513F06E
:106B000045C512F044C511F043C510F066C517F035
:106B100065C516F064C515F063C514F00AEC03F002
:106B20000108D8B4AEEF35F048EC36F076C513F076
:106B300075C512F074C511F073C510F046C517F095
:106B400045C516F044C515F043C514F00AEC03F032
:106B50000108D8B4AEEF35F014EC37F0120004EEB3
:106B6000A4F0140EF76E7A0EF66ED9EC02F0020E57
:106B7000016E5AC52FF059C52EF058C52DF057C5D6
:106B80002CF0030EFEEC00F0140EF76EA60EF66E5F
:106B9000D9EC02F0020E016E3AC52FF039C52EF085
:106BA00038C52DF037C52CF0030EFEEC00F0760E44
:106BB000EE6E2E0EEE6EEF6A28EC1EF0640E24ECE4
:106BC00002F0120004EEA4F0140EF76EB40EF66E8E
:106BD000D9EC02F0020E016E5EC52FF05DC52EF0FD
:106BE0005CC52DF05BC52CF0030EFEEC00F0140E1E
:106BF000F76EE00EF66ED9EC02F0020E016E3EC5A5
:106C00002FF03DC52EF03CC52DF03BC52CF0030EFA
:106C1000FEEC00F0760EEE6E2E0EEE6EEF6A28ECB5
:106C20001EF0640E24EC02F0120004EEA4F0140E28
:106C3000F76EEE0EF66ED9EC02F0020E016E62C532
:106C40002FF061C52EF060C52DF05FC52CF0030E4E
:106C5000FEEC00F0150EF76E1A0EF66ED9EC02F08F
:106C6000020E016E42C52FF041C52EF040C52DF039
:106C70003FC52CF0030EFEEC00F0760EEE6E2E0EED
:106C8000EE6EEF6A28EC1EF0640E24EC02F01200A7
:106C900004EEA4F0150EF76E280EF66ED9EC02F095
:106CA000020E016E66C52FF065C52EF064C52DF08D
:106CB00063C52CF0030EFEEC00F0150EF76E540EBB
:106CC000F66ED9EC02F0020E016E46C52FF045C5F6
:106CD0002EF044C52DF043C52CF0030EFEEC00F061
:106CE000760EEE6E2E0EEE6EEF6A28EC1EF0640E3F
:106CF00024EC02F0120004EEA4F0150EF76E620E02
:106D0000F66ED9EC02F0020E016E6AC52FF069C56D
:106D10002EF068C52DF067C52CF0030EFEEC00F0D8
:106D2000150EF76E8E0EF66ED9EC02F0020E016EA5
:106D30003AC52FF039C52EF038C52DF037C52CF0E7
:106D4000030EFEEC00F0760EEE6E2E0EEE6EEF6A87
:106D500028EC1EF0640E24EC02F0120004EEA4F005
:106D6000150EF76E9C0EF66ED9EC02F0020E016E57
:106D70006EC52FF06DC52EF06CC52DF06BC52CF0D7
:106D8000030EFEEC00F0150EF76EC80EF66ED9EC91
:106D900002F0020E016E3EC52FF03DC52EF03CC53F
:106DA0002DF03BC52CF0030EFEEC00F0760EEE6EDF
:106DB0002E0EEE6EEF6A28EC1EF0640E24EC02F04C
:106DC000120004EEA4F0150EF76ED60EF66ED9EC96
:106DD00002F0020E016E72C52FF071C52EF070C563
:106DE0002DF06FC52CF0030EFEEC00F0160EF76EC2
:106DF000020EF66ED9EC02F0020E016E42C52FF0C3
:106E000041C52EF040C52DF03FC52CF0030EFEEC21
:106E100000F0760EEE6E2E0EEE6EEF6A28EC1EF08F
:106E2000640E24EC02F0120004EEA4F0160EF76ECD
:106E3000100EF66ED9EC02F0020E016E76C52FF040
:106E400075C52EF074C52DF073C52CF0030EFEEC45
:106E500000F0160EF76E3C0EF66ED9EC02F0020E44
:106E6000016E46C52FF045C52EF044C52DF043C533
:106E70002CF0030EFEEC00F0760EEE6E2E0EEE6E93
:106E8000EF6A28EC1EF0640E24EC02F01200160EDD
:106E9000F76E4A0EF66E01EE31F001EC03F0D8A465
:106EA00060EF37F00501776B04EEA4F0160EF76E75
:106EB0004E0EF66ED9EC02F0EF6A000128EC1EF0DF
:106EC000160EF76E6E0EF66E01EE31F001EC03F069
:106ED000D8A47AEF37F0010E0501776F04EEA4F025
:106EE000160EF76E720EF66ED9EC02F0EF6A000124
:106EF00028EC1EF0160EF76E960EF66E01EE31F0CF
:106F000001EC03F0D8A494EF37F0020E0501776F7F
:106F100004EEA4F0160EF76E9E0EF66ED9EC02F09B
:106F2000EF6A000128EC1EF01200010E0501775DEA
:106F30000001D8A4BAEF37F03AC513F039C512F002
:106F400038C511F037C510F03EC517F03DC516F035
:106F50003CC515F03BC514F042EC03F00108D8B471
:106F6000B7EF37F0060109830001B9EF37F00601EA
:106F700009930001020E0501775D0001D8A4F2EF2C
:106F800037F03EC513F03DC512F03CC511F03BC5CE
:106F900010F07BC517F07AC516F079C515F078C5E5
:106FA00014F00AEC03F0356E3EC513F03DC512F047
:106FB0003CC511F03BC510F03AC517F039C516F0C5
:106FC00038C515F037C514F00AEC03F03510D8B405
:106FD000EFEF37F0060109830001F1EF37F006010A
:106FE00009930001120001EE31F084EC00F020C0A2
:106FF00010F021C011F022C012F023C013F0D2EC27
:1070000004F013C07BF512C07AF511C079F510C0F9
:1070100078F51200120001011B6B00019EAA13EF0C
:1070200038F0AECF1BF112009EB818EF38F0FCD745
:107030001BC1ADFF120094928282D8960101D9A1A2
:10704000D8860001D8B631EF38F0160EF76ECE0EA6
:10705000F66ED7EC01F00D0EDFEC01F00A0EDFEC5E
:1070600001F0D896060109ABD8860001D8B684EFA6
:1070700039F081A83EEF38F0ACEF3DF0E86A80BA15
:10708000010E356EE86A81B6010E3510D8B44BEFAB
:1070900038F020EF3CF0D8960501E6A9D88600012B
:1070A000D8B670EF38F00101CE6B010ECD6F000144
:1070B0000101CD510601035D0101CE5106010459C4
:1070C0000001D8A06EEF38F0010E24EC02F00101AF
:1070D000CD2BD8B4CE2B0001D8A4E9D793948194BA
:1070E000060101510501EB5D060102510501EC5954
:1070F0000001D8B07EEF38F03EEC26F081A883EF97
:1071000038F0ACEF3DF0E86A80BA010E356EE86AFF
:1071100081B6010E3510D8B490EF38F0DEEF3BF0B9
:10712000D8960501E6ABD8860001D8B6B5EF38F0A1
:107130000101CE6B010ECD6F00010101CD510601A1
:10714000015D0101CE51060102590001D8A0B3EF43
:1071500038F0010E24EC02F00101CD2BD8B4CE2B77
:107160000001D8A4E9D7939281920501FF51EB5D0C
:10717000060100510501EC590001D8B0C2EF38F00A
:107180003EEC26F081A8C7EF38F0ACEF3DF0E86A9E
:1071900080BA010E356EE86A81B6010E3510D8B49A
:1071A000D4EF38F09CEF3BF0D8960501E6ADD886D9
:1071B0000001D8B6F9EF38F00101CE6B010ECD6FAA
:1071C00000010101CD510501FF5D0101CE51060114
:1071D00000590001D8A0F7EF38F0010E24EC02F0BE
:1071E0000101CD2BD8B4CE2B0001D8A4E9D79390C0
:1071F00081900501FD51EB5DFE51EC590001D8B0C5
:1072000004EF39F03EEC26F081A809EF39F0ACEF3D
:107210003DF0E86A80BA010E356EE86A81B6010E6B
:107220003510D8B416EF39F05AEF3BF0D896050177
:10723000E6AFD8860001D8B63BEF39F00101CE6B3E
:10724000010ECD6F00010101CD510501FD5D010170
:10725000CE510501FE590001D8A039EF39F0010ED9
:1072600024EC02F00101CD2BD8B4CE2B0001D8A420
:10727000E9D7949A829A0501FB51EB5DFC51EC59D8
:107280000001D8B046EF39F03EEC26F081A84BEF74
:1072900039F0ACEF3DF0E86A80BA010E356EE86A6D
:1072A00081B6010E3510D8B458EF39F018EF3BF025
:1072B000D896060109A1D8860001D8B67DEF39F02D
:1072C0000101CE6B010ECD6F00010101CD51050111
:1072D000FB5D0101CE510501FC590001D8A07BEFF7
:1072E00039F0010E24EC02F00101CD2BD8B4CE2BE5
:1072F0000001D8A4E9D79498829881A882EF39F048
:10730000ACEF3DF0D0EF3AF081A889EF39F0ACEF67
:107310003DF0E86A80BA010E356EE86A81B6010E6A
:107320003510D8B496EF39F065EF3DF0D8960501E9
:10733000E6A9D8860001D8B6BBEF39F00101CE6BC3
:10734000010ECD6F00010101CD510501FB5D010171
:10735000CE510501FC590001D8A0B9EF39F0010E5A
:1073600024EC02F00101CD2BD8B4CE2B0001D8A41F
:10737000E9D7949882980501FD51EB5DFE51EC59D7
:107380000001D8B0C6EF39F03EEC26F081A8CBEF73
:1073900039F0ACEF3DF0E86A80BA010E356EE86A6C
:1073A00081B6010E3510D8B4D8EF39F023EF3DF097
:1073B000D8960501E6ABD8860001D8B6FDEF39F0C6
:1073C0000101CE6B010ECD6F00010101CD51050110
:1073D000FD5D0101CE510501FE590001D8A0FBEF72
:1073E00039F0010E24EC02F00101CD2BD8B4CE2BE4
:1073F0000001D8A4E9D7949A829A0501FF51EB5D68
:10740000060100510501EC590001D8B00AEF3AF02D
:107410003EEC26F081A80FEF3AF0ACEF3DF0E86AC1
:1074200080BA010E356EE86A81B6010E3510D8B407
:107430001CEF3AF0E1EF3CF0D8960501E6ADD886B6
:107440000001D8B641EF3AF00101CE6B010ECD6FCD
:1074500000010101CD510501FF5D0101CE51060181
:1074600000590001D8A03FEF3AF0010E24EC02F0E1
:107470000101CD2BD8B4CE2B0001D8A4E9D793902D
:107480008190060101510501EB5D060102510501E4
:10749000EC590001D8B04FEF3AF03EEC26F081A84D
:1074A00054EF3AF0ACEF3DF0E86A80BA010E356E69
:1074B000E86A81B6010E3510D8B461EF3AF09FEF5B
:1074C0003CF0D8960501E6AFD8860001D8B686EF25
:1074D0003AF00101CE6B010ECD6F00010101CD51DB
:1074E0000601015D0101CE51060102590001D8A03B
:1074F00084EF3AF0010E24EC02F00101CD2BD8B458
:10750000CE2B0001D8A4E9D79392819206010351B2
:107510000501EB5D060104510501EC590001D8B0ED
:1075200094EF3AF03EEC26F081A899EF3AF0ACEFF8
:107530003DF0E86A80BA010E356EE86A81B6010E48
:107540003510D8B4A6EF3AF05DEF3CF0D8960601BE
:1075500009A1D8860001D8B6CBEF3AF00101CE6B75
:10756000010ECD6F00010101CD510601035D010146
:10757000CE51060104590001D8A0C9EF3AF0010E1E
:1075800024EC02F00101CD2BD8B4CE2B0001D8A4FD
:10759000E9D79394819481A8D0EF3AF0ACEF3DF015
:1075A00005012A9DD896060109B7D8860001D8B6EC
:1075B000DCEF3AF03EEC26F0EDEF17F0D89606013E
:1075C00009A3D8860001D8B6E8EF3AF0EDEF17F03E
:1075D00094928282D8960101D9A1D8860001D8B6AA
:1075E000FEEF3AF0160EF76EE60EF66ED7EC01F0EF
:1075F0000D0EDFEC01F00A0EDFEC01F0D89606016B
:1076000009A9D8860001D8B64CEF3CF081A80BEF51
:107610003BF0ACEF3DF0010E80BAE86A356E010E2A
:1076200081B6E86A3514D8B418EF3BF0ACEF3DF002
:10763000D8960501E6A9D8860001D8B63DEF3BF003
:107640000101CE6B010ECD6F00010101CD5105018D
:10765000ED5D0101CE510501EE590001D8A03BEFCF
:107660003BF0010E24EC02F00101CD2BD8B4CE2B5F
:107670000001D8A4E9D7949882880501EF51EB5D09
:10768000F051EC590001D8B048EF3BF03EEC26F049
:1076900081A84DEF3BF0ACEF3DF0010E80BAE86AF7
:1076A000356E010E81B6E86A3514D8B45AEF3BF056
:1076B00016EF39F0D8960501E6ABD8860001D8B6AA
:1076C0007FEF3BF00101CE6B010ECD6F0001010198
:1076D000CD510501EF5D0101CE510501F0590001C9
:1076E000D8A07DEF3BF0010E24EC02F00101CD2B80
:1076F000D8B4CE2B0001D8A4E9D7949A828A050188
:10770000F151EB5DF251EC590001D8B08AEF3BF03A
:107710003EEC26F081A88FEF3BF0ACEF3DF0010E80
:1077200080BAE86A356E010E81B6E86A3514D8B4BD
:107730009CEF3BF0D4EF38F0D8960501E6ADD88643
:107740000001D8B6C1EF3BF00101CE6B010ECD6F49
:1077500000010101CD510501F15D0101CE5105018D
:10776000F2590001D8A0BFEF3BF0010E24EC02F06B
:107770000101CD2BD8B4CE2B0001D8A4E9D793902A
:1077800081800501F351EB5DF451EC590001D8B053
:10779000CCEF3BF03EEC26F081A8D1EF3BF0ACEF14
:1077A0003DF0010E80BAE86A356E010E81B6E86AD6
:1077B0003514D8B4DEEF3BF090EF38F0D8960501E1
:1077C000E6AFD8860001D8B603EF3CF00101CE6BDE
:1077D000010ECD6F00010101CD510501F35D0101E5
:1077E000CE510501F4590001D8A001EF3CF0010E83
:1077F00024EC02F00101CD2BD8B4CE2B0001D8A48B
:10780000E9D7939281820501F551EB5DF651EC5970
:107810000001D8B00EEF3CF03EEC26F081A813EF4B
:107820003CF0ACEF3DF0010E80BAE86A356E010E17
:1078300081B6E86A3514D8B420EF3CF04BEF38F04D
:10784000D896060109A1D8860001D8B645EF3CF0CC
:107850000101CE6B010ECD6F00010101CD5105017B
:10786000F55D0101CE510501F6590001D8A043EFA5
:107870003CF0010E24EC02F00101CD2BD8B4CE2B4C
:107880000001D8A4E9D79394818481A84AEF3CF001
:10789000ACEF3DF08FEF3DF081A851EF3CF0ACEF45
:1078A0003DF0010E80BAE86A356E010E81B6E86AD5
:1078B0003514D8B45DEF3CF049D6D8960501E6A959
:1078C000D8860001D8B682EF3CF00101CE6B010EE4
:1078D000CD6F00010101CD510501F55D0101CE51D2
:1078E0000501F6590001D8A080EF3CF0010E24EC10
:1078F00002F00101CD2BD8B4CE2B0001D8A4E9D7DA
:10790000939481840501F351EB5DF451EC5900012E
:10791000D8B08DEF3CF03EEC26F081A892EF3CF021
:10792000ACEF3DF0010E80BAE86A356E010E81B60B
:10793000E86A3514D8B49FEF3CF061EF3AF0D8967E
:107940000501E6ABD8860001D8B6C4EF3CF00101D2
:10795000CE6B010ECD6F00010101CD510501F35D2C
:107960000101CE510501F4590001D8A0C2EF3CF04D
:10797000010E24EC02F00101CD2BD8B4CE2B000176
:10798000D8A4E9D7939281820501F151EB5DF251C0
:10799000EC590001D8B0CFEF3CF03EEC26F081A8C6
:1079A000D4EF3CF0ACEF3DF0010E80BAE86A356EE2
:1079B000010E81B6E86A3514D8B4E1EF3CF01CEF53
:1079C0003AF0D8960501E6ADD8860001D8B606EFA4
:1079D0003DF00101CE6B010ECD6F00010101CD51D3
:1079E0000501F15D0101CE510501F2590001D8A058
:1079F00004EF3DF0010E24EC02F00101CD2BD8B4D0
:107A0000CE2B0001D8A4E9D7939081800501EF51D6
:107A1000EB5DF051EC590001D8B011EF3DF03EECB8
:107A200026F081A816EF3DF0ACEF3DF0010E80BAD4
:107A3000E86A356E010E81B6E86A3514D8B423EFD2
:107A40003DF0D8EF39F0D8960501E6AFD8860001B1
:107A5000D8B648EF3DF00101CE6B010ECD6F0001AD
:107A60000101CD510501EF5D0101CE510501F05934
:107A70000001D8A046EF3DF0010E24EC02F0010118
:107A8000CD2BD8B4CE2B0001D8A4E9D7949A828A02
:107A90000501ED51EB5DEE51EC590001D8B053EF0B
:107AA0003DF03EEC26F081A858EF3DF0ACEF3DF004
:107AB000010E80BAE86A356E010E81B6E86A3514A7
:107AC000D8B465EF3DF096EF39F0D896060109A1DC
:107AD000D8860001D8B68AEF3DF00101CE6B010EC9
:107AE000CD6F00010101CD510501ED5D0101CE51C8
:107AF0000501EE590001D8A088EF3DF0010E24ECFD
:107B000002F00101CD2BD8B4CE2B0001D8A4E9D7C7
:107B10009498828881A88FEF3DF0ACEF3DF005018D
:107B20002A8DD896060109B7D8860001D8B69BEFF2
:107B30003DF03EEC26F0EDEF17F005012A9D000127
:107B4000EDEF17F005012A8D000181A8AAEF3DF0A5
:107B5000ACEF3DF0EDEF17F09DEC2AF0EDEF17F0F4
:107B6000160EF76EFC0EF66E01EE31F001EC03F02E
:107B7000D8A4BEEF3DF0010E01016B6F0001170E9E
:107B8000F76E040EF66E01EE31F001EC03F0D8A4AE
:107B9000D8EF3DF001016B6B04EEA4F0170EF76E09
:107BA0000C0EF66ED9EC02F0EF6A000128EC1EF024
:107BB0001200170EF76E220EF66E01EE31F001EC98
:107BC00003F0D8A4ECEF3DF006010987010E010196
:107BD000686F0001FCEF3DF0060109970101686B39
:107BE00004EEA4F0170EF76E260EF66ED9EC02F036
:107BF000EF6A000128EC1EF01200170EF76E360E29
:107C0000F66E01EE31F001EC03F0D8A40DEF3EF07A
:107C1000060109970101686B696B0001170EF76E89
:107C20003C0EF66E01EE31F001EC03F0D8A420EF2B
:107C30003EF006010987010E0101686F010E696FB0
:107C40000001120005EED0F011EE31F0060EE6CF85
:107C5000EEFFE82EFCD7EF6A04EEA4F0170EF76EE5
:107C6000440EF66ED9EC02F015EED0F0060EE75297
:107C700004E0E6CFEEFFE82EFAD7EF6A28EC1EF01C
:107C8000120005EE92F015EED0F0060EE75204E079
:107C9000E6CFEEFFE82EFAD7EF6A81EC2BF0120068
:107CA00004EEA4F0170EF76E560EF66ED9EC02F045
:107CB00011EE31F0360EE75204E0E6CFEEFFE82E8B
:107CC000FAD7EF6A28EC1EF001EE31F084EC00F0F8
:107CD0000501D86F21C0D9F50001120004EEA4F00F
:107CE000170EF76E6C0EF66ED9EC02F011EE31F055
:107CF000360EE75204E0E6CFEEFFE82EFAD7EF6A41
:107D000028EC1EF001EE31F084EC00F00501DA6F92
:107D100021C0DBF5000112000AEC38F004EEA4F0FB
:107D2000170EF76E840EF66ED9EC02F0020E016E9D
:107D30000501E551CCEC00F0EF6A000128EC1EF0E3
:107D4000120004EEA4F0170EF76E9C0EF66ED9EC3E
:107D500002F011EE31F0360EE75204E0E6CFEEFF0E
:107D6000E82EFAD72E0EEE6EEF6A28EC1EF001EE2A
:107D700031F084EC00F00501E56F0001120004EE23
:107D8000A4F0170EF76EB80EF66ED9EC02F011EEF5
:107D900031F0360EE75204E0E6CFEEFFE82EFAD7D8
:107DA000200EEE6E6D0EEE6E730EEE6E2E0EEE6EFD
:107DB000EF6A28EC1EF001EE31F084EC00F00501D2
:107DC000ED6F21C0EEF50001120004EEA4F0170ED5
:107DD000F76ECE0EF66ED9EC02F011EE31F0360EE3
:107DE000E75204E0E6CFEEFFE82EFAD7200EEE6E63
:107DF0006D0EEE6E730EEE6E2E0EEE6EEF6A28ECCA
:107E00001EF001EE31F084EC00F00501EF6F21C0AF
:107E1000F0F50001120004EEA4F0170EF76EE40E68
:107E2000F66ED9EC02F011EE31F0360EE75204E0B6
:107E3000E6CFEEFFE82EFAD7200EEE6E6D0EEE6E58
:107E4000730EEE6E2E0EEE6EEF6A28EC1EF001EE53
:107E500031F084EC00F00501F16F21C0F2F5000172
:107E6000120004EEA4F0170EF76EFA0EF66ED9ECBF
:107E700002F011EE31F0360EE75204E0E6CFEEFFED
:107E8000E82EFAD7200EEE6E6D0EEE6E730EEE6ECD
:107E90002E0EEE6EEF6A28EC1EF001EE31F084EC4F
:107EA00000F00501F36F21C0F4F50001120004EEAB
:107EB000A4F0180EF76E100EF66ED9EC02F011EE6B
:107EC00031F0360EE75204E0E6CFEEFFE82EFAD7A7
:107ED000200EEE6E6D0EEE6E730EEE6E2E0EEE6ECC
:107EE000EF6A28EC1EF001EE31F084EC00F00501A1
:107EF000F56F21C0F6F50001120004EEA4F0180E93
:107F0000F76E260EF66ED9EC02F011EE31F0360E59
:107F1000E75204E0E6CFEEFFE82EFAD7200EEE6E31
:107F20006D0EEE6E730EEE6E2E0EEE6EEF6A28EC98
:107F30001EF001EE31F084EC00F00501FB6F21C072
:107F4000FCF50001120004EEA4F0180EF76E3A0ED4
:107F5000F66ED9EC02F011EE31F0360EE75204E085
:107F6000E6CFEEFFE82EFAD7200EEE6E6D0EEE6E27
:107F7000730EEE6E2E0EEE6EEF6A28EC1EF001EE22
:107F800031F084EC00F00501FD6F21C0FEF5000129
:107F9000120004EEA4F0180EF76E4E0EF66ED9EC39
:107FA00002F011EE31F0360EE75204E0E6CFEEFFBC
:107FB000E82EFAD7200EEE6E6D0EEE6E730EEE6E9C
:107FC0002E0EEE6EEF6A28EC1EF001EE31F084EC1E
:107FD00000F00501FF6F21C000F60001120004EE61
:107FE000A4F0180EF76E620EF66ED9EC02F011EEE8
:107FF00031F0360EE75204E0E6CFEEFFE82EFAD776
:10800000200EEE6E6D0EEE6E730EEE6E2E0EEE6E9A
:10801000EF6A28EC1EF001EE31F084EC00F006016E
:10802000016F21C002F60001120004EEA4F0180E48
:10803000F76E760EF66ED9EC02F011EE31F0360ED8
:10804000E75204E0E6CFEEFFE82EFAD7200EEE6E00
:108050006D0EEE6E730EEE6E2E0EEE6EEF6A28EC67
:108060001EF001EE31F084EC00F00601036F21C038
:1080700004F600011200310E0101315D0001D8A4A7
:1080800049EF40F00501E68901EEA0F0310EEE6EF9
:10809000EF6A0001320E0101315D0001D8A458EFF2
:1080A00040F00501E68B01EEA0F0320EEE6EEF6AB5
:1080B0000001330E0101315D0001D8A467EF40F0EB
:1080C0000501E68D01EEA0F0330EEE6EEF6A0001C1
:1080D000340E0101315D0001D8A476EF40F00501B6
:1080E000E68F01EEA0F0340EEE6EEF6A0001350E61
:1080F0000101315D0001D8A485EF40F0060109813E
:1081000001EEA0F0350EEE6EEF6A000104EEA4F071
:10811000180EF76E8A0EF66ED9EC02F011EEA0F092
:10812000140EE75204E0E6CFEEFFE82EFAD7180E61
:10813000F76E920EF66ED9EC02F0EF6A28EC1EF0A4
:108140001200310E0101315D0001D8A4AFEF40F003
:108150000501E69901EEA0F0310EEE6EEF6A000126
:10816000320E0101315D0001D8A4BEEF40F00501DF
:10817000E69B01EEA0F0320EEE6EEF6A0001330EC8
:108180000101315D0001D8A4CDEF40F00501E69D6D
:1081900001EEA0F0330EEE6EEF6A0001340E010125
:1081A000315D0001D8A4DCEF40F00501E69F01EE4F
:1081B000A0F0340EEE6EEF6A0001350E0101315D64
:1081C0000001D8A4EBEF40F00601099101EEA0F008
:1081D000350EEE6EEF6A000104EEA4F0180EF76E95
:1081E0009C0EF66ED9EC02F011EEA0F0140EE752E0
:1081F00004E0E6CFEEFFE82EFAD7180EF76EA40ED5
:10820000F66ED9EC02F0EF6A28EC1EF01200180EA0
:10821000F76EAE0EF66E01EE31F001EC03F0D8A46D
:1082200013EF41F08288180EF76EB20EF66E01EE73
:1082300031F001EC03F0D8A41FEF41F0829882A83E
:108240002DEF41F004EEA4F0180EF76EB60EF66EA8
:10825000D9EC02F0EF6A28EC1EF082B83BEF41F057
:1082600004EEA4F0180EF76EC80EF66ED9EC02F00C
:10827000EF6A28EC1EF01200180EF76EDA0EF66E9A
:1082800001EE31F001EC03F0D8A448EF41F0828A0E
:10829000180EF76EDE0EF66E01EE31F001EC03F013
:1082A000D8A454EF41F0829A82AA62EF41F004EE22
:1082B000A4F0180EF76EE20EF66ED9EC02F0EF6A3B
:1082C00028EC1EF082BA70EF41F004EEA4F0180E14
:1082D000F76EF40EF66ED9EC02F0EF6A28EC1EF0A1
:1082E0001200190EF76E060EF66E01EE31F001EC7B
:1082F00003F0D8A47DEF41F08180190EF76E0A0ECD
:10830000F66E01EE31F001EC03F0D8A489EF41F0F4
:10831000819081A097EF41F004EEA4F0190EF76E62
:108320000E0EF66ED9EC02F0EF6A28EC1EF081B06A
:10833000A5EF41F004EEA4F0190EF76E200EF66ED4
:10834000D9EC02F0EF6A28EC1EF01200190EF76E5D
:10835000320EF66E01EE31F001EC03F0D8A4B2EF6C
:1083600041F08182190EF76E360EF66E01EE31F095
:1083700001EC03F0D8A4BEEF41F0819281A2CCEFD2
:1083800041F004EEA4F0190EF76E3A0EF66ED9EC39
:1083900002F0EF6A28EC1EF081B2DAEF41F004EE51
:1083A000A4F0190EF76E4C0EF66ED9EC02F0EF6ADF
:1083B00028EC1EF01200190EF76E5E0EF66E01EE3E
:1083C00031F001EC03F0D8A4E7EF41F08184190EFD
:1083D000F76E620EF66E01EE31F001EC03F0D8A4F8
:1083E000F3EF41F0819481A401EF42F004EEA4F098
:1083F000190EF76E660EF66ED9EC02F0EF6A28ECF5
:108400001EF081B40FEF42F004EEA4F0190EF76EE7
:10841000780EF66ED9EC02F0EF6A28EC1EF012002E
:10842000120012001200190EF76E8A0EF66E01EE9F
:1084300031F001EC03F0D8A420EF42F006010B8FDD
:108440000001190EF76E8E0EF66E01EE31F001ECA2
:1084500003F0D8A42EEF42F006010B9F0001D8963E
:1084600006010BAFD8860001D8B642EF42F004EE09
:10847000A4F0190EF76E920EF66ED9EC02F0EF6AC8
:1084800028EC1EF0D89606010BBFD8860001D8B69E
:1084900055EF42F004EEA4F0190EF76EA20EF66E40
:1084A000D9EC02F0EF6A28EC1EF00601098D0001FC
:1084B0001200190EF76EB40EF66E01EE31F001ECFB
:1084C00003F0D8A466EF42F006010C810001190EFA
:1084D000F76EB80EF66E01EE31F001EC03F0D8A4A1
:1084E00074EF42F006010C910001D89606010CA130
:1084F000D8860001D8B688EF42F004EEA4F0190E39
:10850000F76EBC0EF66ED9EC02F0EF6A28EC1EF0A6
:10851000D89606010CB1D8860001D8B69BEF42F080
:1085200004EEA4F0190EF76ECC0EF66ED9EC02F044
:10853000EF6A28EC1EF00601098D00011200190EE9
:10854000F76EDE0EF66E01EE31F001EC03F0D8A40A
:10855000ACEF42F006010C830001190EF76EE20E3B
:10856000F66E01EE31F001EC03F0D8A4BAEF42F060
:1085700006010C930001D89606010CA3D8860001D1
:10858000D8B6CEEF42F004EEA4F0190EF76EE60E68
:10859000F66ED9EC02F0EF6A28EC1EF0D8960601D0
:1085A0000CB3D8860001D8B6E1EF42F004EEA4F097
:1085B000190EF76EF60EF66ED9EC02F0EF6A28ECA3
:1085C0001EF00601098D00011200310E0101315D1E
:1085D0000001D8A4F1EF42F08288FA0E24EC02F0F8
:1085E0008298320E0101315D0001D8A4FDEF42F006
:1085F000828AFA0E24EC02F0829A330E0101315D78
:108600000001D8A409EF43F08180FA0E24EC02F0B7
:108610008190340E0101315D0001D8A415EF43F0C3
:108620008182FA0E24EC02F08192350E0101315D57
:108630000001D8A421EF43F08184FA0E24EC02F06B
:1086400081940601098D0001120004EEA4F01A0EB7
:10865000F76E080EF66ED9EC02F0EF6A28EC1EF009
:10866000010E0501E56F010EE36FEE6B010EED6F7C
:10867000F06B640EEF6FF26B640EF16FF46B640ECF
:10868000F36FF66B640EF56FF86B640EF76FFA6BB1
:10869000640EF96FFC6B010EFB6FFE6B640EFD6FD9
:1086A0000601006B640E0501FF6F0601026B640E8C
:1086B000016F046B640E036F066B640E056F086B2D
:1086C000640E076F0989098B140E0501906F776B93
:1086D000CD0E7B6FCC0E7A6F4C0E796F7C0E786F5F
:1086E0000601099505014A6B496B486B476B4E6B58
:1086F0004D6B4C6B4B6B526B516B506B4F6B566BA6
:10870000556B546B536B010169530001D8A48BEF77
:1087100043F0ADEC4AF001016B6B686B0601099701
:108720000501256B5A6B596B586B576B5E6B5D6B14
:108730005C6B5B6B626B616B606B5F6B666B656BDD
:10874000646B636B6A6B696B700E686F830E676F27
:108750006E6B6D6B700E6C6F830E6B6F726B716BEB
:10876000700E706F830E6F6F766B756B700E746F1B
:10877000830E736F0401A36B01016C6B0501EC6B3D
:10878000FA0EEB6F00011200010E0501D76FAA6A05
:10879000A96AD751FEEC01F00A0E24EC02F0AA6A95
:1087A000020EA96ED851FEEC01F0D951FEEC01F099
:1087B0000A0E24EC02F0AA6A040EA96EDA51FEEC4D
:1087C00001F0DB51FEEC01F00A0E24EC02F0AA6A83
:1087D000060EA96EE551FEEC01F00A0E24EC02F043
:1087E000AA6A0A0EA96E000EFEEC01F0AA6A140E27
:1087F000A96EED51FEEC01F0EE51FEEC01F00A0E17
:1088000024EC02F0AA6A160EA96EEF51FEEC01F0FC
:10881000F051FEEC01F00A0E24EC02F0AA6A180EE8
:10882000A96EF151FEEC01F0F251FEEC01F00A0EDE
:1088300024EC02F0AA6A1A0EA96EF351FEEC01F0C4
:10884000F451FEEC01F00A0E24EC02F0AA6A1C0EB0
:10885000A96EF551FEEC01F0F651FEEC01F00A0EA6
:1088600024EC02F0AA6A1E0EA96EF751FEEC01F08C
:10887000F851FEEC01F00A0E24EC02F0AA6A200E78
:10888000A96EF951FEEC01F0FA51FEEC01F00A0E6E
:1088900024EC02F0AA6A280EA96EFB51FEEC01F04E
:1088A000FC51FEEC01F00A0E24EC02F0AA6A2A0E3A
:1088B000A96EFD51FEEC01F0FE51FEEC01F00A0E36
:1088C00024EC02F0AA6A2C0EA96EFF51FEEC01F016
:1088D00006010051FEEC01F00A0E24EC02F0AA6A37
:1088E0002E0EA96E0151FEEC01F00251FEEC01F0DA
:1088F0000A0E24EC02F0AA6A300EA96E0351FEECB7
:1089000001F00451FEEC01F00A0E24EC02F0AA6A18
:10891000320EA96E0551FEEC01F00651FEEC01F09D
:108920000A0E24EC02F0AA6A340EA96E0751FEEC7E
:1089300001F00851FEEC01F00A0E24EC02F0AA6AE4
:108940003C0EA96EE86A09B9010EFEEC01F00A0EB0
:1089500024EC02F0AA6A3E0EA96EE86A09BB010E79
:10896000FEEC01F00A0E24EC02F0AA6A400EA96E99
:108970000401A351FEEC01F00A0E24EC02F0AA6AF5
:10898000410EA96E05EED0F0EE5003E0FEEC01F0D2
:10899000FBD70A0E24EC02F001EECAF015EED0F07F
:1089A000010EF36E010EE1EC02F0EF6AAA6A410ECD
:1089B000A96E01EECAF0EE5003E0FEEC01F0FBD729
:1089C0000A0E24EC02F001EECAF015EED0F0020E11
:1089D000F36E010EE1EC02F0EF6AAA6A420EA96E94
:1089E00001EECAF0EE5003E0FEEC01F0FBD70A0EF8
:1089F00024EC02F001EECAF015EED0F0030EF36E97
:108A0000010EE1EC02F0EF6AAA6A430EA96E01EED4
:108A1000CAF0EE5003E0FEEC01F0FBD70A0E24ECA6
:108A200002F001EECAF015EED0F0040EF36E010E66
:108A3000E1EC02F0EF6AAA6A440EA96E01EECAF0F8
:108A4000EE5003E0FEEC01F0FBD70A0E24EC02F03E
:108A500001EECAF015EED0F0050EF36E010EE1EC5A
:108A600002F0EF6AAA6A450EA96E01EECAF0EE5056
:108A700003E0FEEC01F0FBD70A0E24EC02F001EE5D
:108A8000CAF015EED0F0060EF36E010EE1EC02F026
:108A9000EF6AAA6A460EA96E01EECAF0EE5003E034
:108AA000FEEC01F0FBD70A0E24EC02F0AA6A500E8D
:108AB000A96EE86A0501E6B9010EFEEC01F00A0EA6
:108AC00024EC02F0AA6A510EA96EE86AE6BB010E18
:108AD000FEEC01F00A0E24EC02F0AA6A520EA96E16
:108AE000E86AE6BD010EFEEC01F00A0E24EC02F08D
:108AF000AA6A530EA96EE86AE6BF010EFEEC01F009
:108B00000A0E24EC02F0AA6A540EA96EE86A060165
:108B100009B1010EFEEC01F00A0E24EC02F0AA6A83
:108B2000550EA96E05019051FEEC01F00A0E24ECE1
:108B300002F0AA6A560EA96E7751FEEC01F00A0EF9
:108B400024EC02F0AA6A570EA96E7851FEEC01F0EF
:108B50007951FEEC01F07A51FEEC01F07B51FEEC14
:108B600001F00A0E24EC02F0AA6A5B0EA96EE86A14
:108B7000060109B7010EFEEC01F00A0E24EC02F02A
:108B8000AA6A5C0EA96E05014751FEEC01F048513E
:108B9000FEEC01F04951FEEC01F04A51FEEC01F00F
:108BA0000A0E24EC02F0AA6A600EA96E4B51FEEC8C
:108BB00001F04C51FEEC01F04D51FEEC01F04E5134
:108BC000FEEC01F00A0E24EC02F0AA6A640EA96E13
:108BD0004F51FEEC01F05051FEEC01F05151FEEC12
:108BE00001F05251FEEC01F00A0E24EC02F0AA6AE8
:108BF000680EA96E5351FEEC01F05451FEEC01F0E9
:108C00005551FEEC01F05651FEEC01F00A0E24EC39
:108C100002F0AA6A6C0EA96E01016851FEEC01F027
:108C20000A0E24EC02F0AA6A6D0EA96E6951FEECE0
:108C300001F00A0E24EC02F0AA6A6E0EA96E6B51C6
:108C4000FEEC01F00A0E24EC02F0AA6A6F0EA96E87
:108C500005015751FEEC01F05851FEEC01F059515D
:108C6000FEEC01F05A51FEEC01F00A0E24EC02F089
:108C7000AA6A730EA96E5B51FEEC01F05C51FEEC2A
:108C800001F05D51FEEC01F05E51FEEC01F00A0EC8
:108C900024EC02F0AA6A770EA96E5F51FEEC01F097
:108CA0006051FEEC01F06151FEEC01F06251FEEC0E
:108CB00001F00A0E24EC02F0AA6A7B0EA96E635141
:108CC000FEEC01F06451FEEC01F06551FEEC01F0A8
:108CD0006651FEEC01F00A0E24EC02F0AA6A7F0E47
:108CE000A96E6751FEEC01F06851FEEC01F069518C
:108CF000FEEC01F06A51FEEC01F00A0E24EC02F0E9
:108D0000AA6A830EA96E6B51FEEC01F06C51FEEC69
:108D100001F06D51FEEC01F06E51FEEC01F00A0E17
:108D200024EC02F0AA6A870EA96E6F51FEEC01F0E6
:108D30007051FEEC01F07151FEEC01F07251FEEC4D
:108D400001F00A0E24EC02F0AA6A8B0EA96E735190
:108D5000FEEC01F07451FEEC01F07551FEEC01F0F7
:108D60007651FEEC01F00A0E24EC02F0AA6A8F0E96
:108D7000A96E01016C51FEEC01F00A0E24EC02F028
:108D8000AA6A900EA96E05012551FEEC01F00A0EAB
:108D900024EC02F0AA6A910EA96EEB51FEEC01F0F0
:108DA000EC51FEEC01F00A0E24EC02F004EEA4F00B
:108DB0001A0EF76E300EF66ED9EC02F0EF6A000173
:108DC00028EC1EF01200000EF5EC01F00501D76F43
:108DD000020EF5EC01F0D86FF7EC01F0D96F040E3C
:108DE000F5EC01F0DA6FF7EC01F0DB6F060EF5EC55
:108DF00001F0E56F0A0EF5EC01F0E36FE329E46F93
:108E0000140EF5EC01F0ED6FF7EC01F0EE6F160EBD
:108E1000F5EC01F0EF6FF7EC01F0F06F180EF5ECE8
:108E200001F0F16FF7EC01F0F26F1A0EF5EC01F0C2
:108E3000F36FF7EC01F0F46F1C0EF5EC01F0F56F39
:108E4000F7EC01F0F66F1E0EF5EC01F0F76FF7ECA2
:108E500001F0F86F200EF5EC01F0F96FF7EC01F07E
:108E6000FA6F280EF5EC01F0FB6FF7EC01F0FC6FE8
:108E70002A0EF5EC01F0FD6FF7EC01F0FE6F2C0E01
:108E8000F5EC01F0FF6FF7EC01F00601006F2E0E1C
:108E9000F5EC01F0016FF7EC01F0026F300EF5EC2C
:108EA00001F0036FF7EC01F0046F320EF5EC01F006
:108EB000056FF7EC01F0066F340EF5EC01F0076F6B
:108EC000F7EC01F0086F3C0EF5EC01F00989E8A021
:108ED00009993E0EF5EC01F0098BE8A0099B400EC4
:108EE000F5EC01F00401A36F500EF5EC01F0050163
:108EF000E689E8A0E699510EF5EC01F0E68BE8A0D2
:108F0000E69B520EF5EC01F0E68DE8A0E69D530ECF
:108F1000F5EC01F0E68FE8A0E69F540EF5EC01F0C9
:108F200006010981E8A00991550EF5EC01F0050153
:108F3000906F560EF5EC01F0776F570EF5EC01F0DF
:108F4000786FF7EC01F0796FF7EC01F07A6FF7ECDE
:108F500001F07B6F5B0EF5EC01F006010987E8A0DC
:108F600009975C0EF5EC01F00501476FF7EC01F095
:108F7000486FF7EC01F0496FF7EC01F04A6F600EB3
:108F8000F5EC01F04B6FF7EC01F04C6FF7EC01F0F2
:108F90004D6FF7EC01F04E6F640EF5EC01F04F6F82
:108FA000F7EC01F0506FF7EC01F0516FF7EC01F0C6
:108FB000526F680EF5EC01F0536FF7EC01F0546F4F
:108FC000F7EC01F0556FF7EC01F0566F6C0EF5EC15
:108FD00001F00101686F6D0EF5EC01F0696F6E0E26
:108FE000F5EC01F06B6F6F0EF5EC01F00501576FBA
:108FF000F7EC01F0586FF7EC01F0596FF7EC01F066
:109000005A6F730EF5EC01F05B6FF7EC01F05C6FDB
:10901000F7EC01F05D6FF7EC01F05E6F770EF5ECA9
:1090200001F05F6FF7EC01F0606FF7EC01F0616F3A
:10903000F7EC01F0626F7B0EF5EC01F0636FF7EC7B
:1090400001F0646FF7EC01F0656FF7EC01F0666F0B
:109050007F0EF5EC01F0676FF7EC01F0686FF7EC4D
:1090600001F0696FF7EC01F06A6F830EF5EC01F027
:109070006B6FF7EC01F06C6FF7EC01F06D6FF7ECD4
:1090800001F06E6F870EF5EC01F06F6FF7EC01F0F9
:10909000706FF7EC01F0716FF7EC01F0726F8B0EEF
:1090A000F5EC01F0736FF7EC01F0746FF7EC01F081
:1090B000756FF7EC01F0766F8F0EF5EC01F00101A2
:1090C0006C6F900EF5EC01F00501256F910EF5EC3B
:1090D00001F0EB6FF7EC01F0EC6F130EEE5D0001A9
:1090E000D8A081EF48F0D8A47DEF48F0890E0501A3
:1090F000ED5D0001D8A081EF48F00501EE6B320E66
:10910000ED6F000101016B530001D8A48AEF48F014
:10911000ADEC4AF001016B530001D8A49BEF48F07D
:1091200004EEA4F01A0EF76E560EF66ED9EC02F0AD
:10913000EF6A28EC1EF0120004EEA4F01A0EF76E8F
:109140007E0EF66ED9EC02F0EF6A28EC1EF004EE0B
:10915000A4F01A0EF76EBA0EF66ED9EC02F0EF6AB2
:1091600028EC1EF004EEA4F01B0EF76E0C0EF66E4B
:10917000D9EC02F0EF6A28EC1EF004EEA4F01B0E0E
:10918000F76E5E0EF66ED9EC02F0EF6A28EC1EF078
:1091900004EEA4F01B0EF76EA60EF66ED9EC02F0EC
:1091A000EF6A28EC1EF004EEA4F01B0EF76EEE0E34
:1091B000F66ED9EC02F0EF6A28EC1EF004EEA4F093
:1091C0001C0EF76E2C0EF66ED9EC02F0EF6A28EC4E
:1091D0001EF004EEA4F01C0EF76E6A0EF66ED9ECCB
:1091E00002F0EF6A28EC1EF004EEA4F01C0EF76EFD
:1091F000920EF66ED9EC02F0EF6A28EC1EF004EE47
:10920000A4F01C0EF76EBC0EF66ED9EC02F0EF6AFD
:1092100028EC1EF004EEA4F01C0EF76EFA0EF66EAB
:10922000D9EC02F0EF6A28EC1EF004EEA4F01D0E5B
:10923000F76E2A0EF66ED9EC02F0EF6A28EC1EF0FB
:1092400004EEA4F01D0EF76E5E0EF66ED9EC02F081
:10925000EF6A28EC1EF004EEA4F01D0EF76E940EDB
:10926000F66ED9EC02F0EF6A28EC1EF004EEA4F0E2
:109270001D0EF76EC80EF66ED9EC02F0EF6A28EC00
:109280001EF004EEA4F01E0EF76E100EF66ED9EC72
:1092900002F0EF6A28EC1EF004EEA4F01E0EF76E4A
:1092A000340EF66ED9EC02F0EF6A28EC1EF004EEF4
:1092B000A4F01E0EF76E5C0EF66ED9EC02F0EF6AAB
:1092C00028EC1EF004EEA4F01E0EF76E840EF66E6F
:1092D000D9EC02F0EF6A28EC1EF004EEA4F01E0EAA
:1092E000F76ED60EF66ED9EC02F0EF6A28EC1EF09F
:1092F00004EEA4F01F0EF76E140EF66ED9EC02F019
:10930000EF6A28EC1EF004EEA4F01F0EF76E740E48
:10931000F66ED9EC02F0EF6A28EC1EF004EEA4F031
:109320001F0EF76EBC0EF66ED9EC02F0EF6A28EC59
:109330001EF004EEA4F0200EF76E060EF66ED9ECC9
:1093400002F0EF6A28EC1EF004EEA4F0200EF76E97
:10935000360EF66ED9EC02F0EF6A28EC1EF004EE41
:10936000A4F0200EF76E740EF66ED9EC02F0EF6AE0
:1093700028EC1EF004EEA4F0200EF76ED40EF66E6C
:10938000D9EC02F0EF6A28EC1EF004EEA4F0210EF6
:10939000F76E0C0EF66ED9EC02F0EF6A28EC1EF0B8
:1093A00004EEA4F0210EF76E7C0EF66ED9EC02F0FE
:1093B000EF6A28EC1EF004EEA4F0210EF76EC60E44
:1093C000F66ED9EC02F0EF6A28EC1EF004EEA4F081
:1093D000220EF76E040EF66ED9EC02F0EF6A28EC5E
:1093E0001EF004EEA4F0220EF76E560EF66ED9ECC7
:1093F00002F0EF6A28EC1EF004EEA4F0220EF76EE5
:10940000AC0EF66ED9EC02F0EF6A28EC1EF004EE1A
:10941000A4F0220EF76EF00EF66ED9EC02F0EF6AB1
:1094200028EC1EF004EEA4F0230EF76E360EF66E56
:10943000D9EC02F0EF6A28EC1EF004EEA4F0230E43
:10944000F76E740EF66ED9EC02F0EF6A28EC1EF09F
:1094500004EEA4F0230EF76EC00EF66ED9EC02F007
:10946000EF6A28EC1EF004EEA4F0230EF76EFE0E59
:10947000F66ED9EC02F0EF6A28EC1EF004EEA4F0D0
:10948000240EF76E460EF66ED9EC02F0EF6A28EC69
:109490001EF004EEA4F0240EF76E880EF66ED9ECE2
:1094A00002F0EF6A28EC1EF004EEA4F0240EF76E32
:1094B000BC0EF66ED9EC02F0EF6A28EC1EF004EE5A
:1094C000A4F0240EF76EF40EF66ED9EC02F0EF6AFB
:1094D00028EC1EF004EEA4F0250EF76E320EF66EA8
:1094E000D9EC02F0EF6A28EC1EF004EEA4F0250E91
:1094F000F76E640EF66ED9EC02F0EF6A28EC1EF0FF
:1095000004EEA4F0250EF76E960EF66ED9EC02F07E
:10951000EF6A28EC1EF004EEA4F0250EF76ED40ED0
:10952000F66ED9EC02F0EF6A28EC1EF004EEA4F01F
:10953000260EF76E000EF66ED9EC02F0EF6A28ECFC
:109540001EF004EEA4F0260EF76E2E0EF66ED9EC89
:1095500002F0EF6A28EC1EF0120004EEA4F0260ED2
:10956000F76E720EF66ED9EC02F0EF6A28EC1EF080
:1095700001EE6DF0020E016E0501D751CCEC00F04A
:10958000EF6A04EEA4F0260EF76E9A0EF66ED9EC92
:1095900002F011EE6DF0320EE75204E0E6CFEEFF7E
:1095A000E82EFAD7EF6A000128EC1EF001EE6DF00C
:1095B00015EEDCF0060EE75204E0E6CFEEFFE82EF3
:1095C000FAD7EF6A04EEA4F0260EF76EAA0EF66E36
:1095D000D9EC02F011EE6DF0320EE75204E0E6CF66
:1095E000EEFFE82EFAD7EF6A28EC1EF001EE6DF0E0
:1095F000020E016E086AD9C521F0D8C520F0CFEC63
:1096000000F0EF6A04EEA4F0260EF76EBA0EF66EC6
:10961000D9EC02F011EE6DF0320EE75204E0E6CF25
:10962000EEFFE82EFAD7EF6A28EC1EF001EE6DF09F
:10963000020E016E086ADBC521F0DAC520F0CFEC1E
:1096400000F0EF6A04EEA4F0260EF76ECA0EF66E76
:10965000D9EC02F011EE6DF0320EE75204E0E6CFE5
:10966000EEFFE82EFAD7EF6A28EC1EF001EE6DF05F
:10967000020E016E0501E551CCEC00F0EF6A04EE3C
:10968000A4F0260EF76EDA0EF66ED9EC02F011EEAB
:109690006DF0320EE75204E0E6CFEEFFE82EFAD787
:1096A000EF6A000128EC1EF001EE6DF0020E016E73
:1096B000086AEEC521F0EDC520F0CFEC00F0EF6AAE
:1096C00004EEA4F0260EF76EEA0EF66ED9EC02F068
:1096D00011EE6DF0320EE75204E0E6CFEEFFE82E19
:1096E000FAD7EF6A28EC1EF001EE6DF0020E016E63
:1096F000086AF0C521F0EFC520F0CFEC00F0EF6A6A
:1097000004EEA4F0260EF76EFA0EF66ED9EC02F017
:1097100011EE6DF0320EE75204E0E6CFEEFFE82ED8
:10972000FAD7EF6A28EC1EF001EE6DF0020E016E22
:10973000086AF2C521F0F1C520F0CFEC00F0EF6A25
:1097400004EEA4F0270EF76E0A0EF66ED9EC02F0C6
:1097500011EE6DF0320EE75204E0E6CFEEFFE82E98
:10976000FAD7EF6A28EC1EF001EE6DF0020E016EE2
:10977000086AF4C521F0F3C520F0CFEC00F0EF6AE1
:1097800004EEA4F0270EF76E1A0EF66ED9EC02F076
:1097900011EE6DF0320EE75204E0E6CFEEFFE82E58
:1097A000FAD7EF6A28EC1EF001EE6DF0020E016EA2
:1097B000086AF6C521F0F5C520F0CFEC00F0EF6A9D
:1097C00004EEA4F0270EF76E2A0EF66ED9EC02F026
:1097D00011EE6DF0320EE75204E0E6CFEEFFE82E18
:1097E000FAD7EF6A28EC1EF001EE6DF0020E016E62
:1097F000086AFCC521F0FBC520F0CFEC00F0EF6A51
:1098000004EEA4F0270EF76E3A0EF66ED9EC02F0D5
:1098100011EE6DF0320EE75204E0E6CFEEFFE82ED7
:10982000FAD7EF6A28EC1EF001EE6DF0020E016E21
:10983000086AFEC521F0FDC520F0CFEC00F0EF6A0C
:1098400004EEA4F0270EF76E4A0EF66ED9EC02F085
:1098500011EE6DF0320EE75204E0E6CFEEFFE82E97
:10986000FAD7EF6A28EC1EF001EE6DF0020E016EE1
:10987000086A00C621F0FFC520F0CFEC00F0EF6AC7
:1098800004EEA4F0270EF76E5A0EF66ED9EC02F035
:1098900011EE6DF0320EE75204E0E6CFEEFFE82E57
:1098A000FAD7EF6A28EC1EF001EE6DF0020E016EA1
:1098B000086A02C621F001C620F0CFEC00F0EF6A82
:1098C00004EEA4F0270EF76E6A0EF66ED9EC02F0E5
:1098D00011EE6DF0320EE75204E0E6CFEEFFE82E17
:1098E000FAD7EF6A28EC1EF001EE6DF0020E016E61
:1098F000086A04C621F003C620F0CFEC00F0EF6A3E
:1099000004EEA4F0270EF76E7A0EF66ED9EC02F094
:1099100011EE6DF0320EE75204E0E6CFEEFFE82ED6
:10992000FAD7EF6A28EC1EF0D8960501E6A9D8868A
:109930000001D8B6A7EF4CF001EEA0F0270EF76EAD
:109940008A0EF66ED9EC02F0EF6AB0EF4CF001EE41
:10995000A0F0270EF76E940EF66ED9EC02F0EF6AC7
:1099600004EEA4F0270EF76EA00EF66ED9EC02F00E
:1099700011EEA0F0140EE75204E0E6CFEEFFE82E61
:10998000FAD7EF6A28EC1EF0D8960501E6ABD88628
:109990000001D8B6D7EF4CF001EEA0F0270EF76E1D
:1099A000AE0EF66ED9EC02F0EF6AE0EF4CF001EE8D
:1099B000A0F0270EF76EB80EF66ED9EC02F0EF6A43
:1099C00004EEA4F0270EF76EC40EF66ED9EC02F08A
:1099D00011EEA0F0140EE75204E0E6CFEEFFE82E01
:1099E000FAD7EF6A28EC1EF0D8960501E6ADD886C6
:1099F0000001D8B607EF4DF001EEA0F0270EF76E8C
:109A0000D20EF66ED9EC02F0EF6A10EF4DF001EED7
:109A1000A0F0270EF76EDC0EF66ED9EC02F0EF6ABE
:109A200004EEA4F0270EF76EE80EF66ED9EC02F005
:109A300011EEA0F0140EE75204E0E6CFEEFFE82EA0
:109A4000FAD7EF6A28EC1EF0D8960501E6AFD88663
:109A50000001D8B637EF4DF001EEA0F0270EF76EFB
:109A6000F60EF66ED9EC02F0EF6A40EF4DF001EE23
:109A7000A0F0280EF76E000EF66ED9EC02F0EF6A39
:109A800004EEA4F0280EF76E0C0EF66ED9EC02F080
:109A900011EEA0F0140EE75204E0E6CFEEFFE82E40
:109AA000FAD7EF6A28EC1EF0D896060109A1D886ED
:109AB0000001D8B667EF4DF001EEA0F0280EF76E6A
:109AC0001A0EF66ED9EC02F0EF6A70EF4DF001EE6F
:109AD000A0F0280EF76E240EF66ED9EC02F0EF6AB5
:109AE00004EEA4F0280EF76E300EF66ED9EC02F0FC
:109AF00011EEA0F0140EE75204E0E6CFEEFFE82EE0
:109B0000FAD7EF6A28EC1EF0D896060109A9D88684
:109B10000001D8B699EF4DF004EEA4F0280EF76ED0
:109B20003E0EF66ED9EC02F0EF6A28EC1EF0A4EFC0
:109B30004DF004EEA4F0280EF76E540EF66ED9EC3C
:109B400002F0EF6A28EC1EF0D896060109ABD88621
:109B50000001D8B6B9EF4DF004EEA4F0280EF76E70
:109B60006C0EF66ED9EC02F0EF6A28EC1EF0C4EF32
:109B70004DF004EEA4F0280EF76E820EF66ED9ECCE
:109B800002F0EF6A28EC1EF004EEA4F0280EF76E47
:109B90009A0EF66ED9EC02F0020E016E050190519C
:109BA000CCEC00F0EF6A000128EC1EF005017753C1
:109BB0000001D8A4E5EF4DF004EEA4F0280EF76EF6
:109BC000AA0EF66ED9EC02F0EF6A010E0501775D80
:109BD0000001D8A4F5EF4DF004EEA4F0280EF76EC6
:109BE000C20EF66ED9EC02F0EF6A020E0501775D47
:109BF0000001D8A412EF4EF004EEA4F0280EF76E88
:109C0000E60EF66ED9EC02F0020E016E7BC52FF067
:109C10007AC52EF079C52DF078C52CF0030EFEEC38
:109C200000F0EF6A01016C530001D8A423EF4EF05D
:109C300004EEA4F0290EF76E000EF66ED9EC02F0D9
:109C4000EF6A28EC1EF0010E01016C5D0001D8A442
:109C500035EF4EF004EEA4F0290EF76E140EF66EFA
:109C6000D9EC02F0EF6A28EC1EF001EE6DF0020E66
:109C7000016E5AC52FF059C52EF058C52DF057C5A5
:109C80002CF0030EFEEC00F0EF6A04EEA4F0290EB7
:109C9000F76E260EF66ED9EC02F011EE6DF0320E74
:109CA000E75204E0E6CFEEFFE82EFAD7EF6A28ECA1
:109CB0001EF001EE6DF0020E016E6AC52FF069C54F
:109CC0002EF068C52DF067C52CF0030EFEEC00F0F9
:109CD000EF6A04EEA4F0290EF76E360EF66ED9EC9C
:109CE00002F011EE6DF0320EE75204E0E6CFEEFF27
:109CF000E82EFAD7EF6A28EC1EF001EE6DF0020EA6
:109D0000016E4AC52FF049C52EF048C52DF047C554
:109D10002CF0030EFEEC00F0EF6A04EEA4F0290E26
:109D2000F76E460EF66ED9EC02F011EE6DF0320EC3
:109D3000E75204E0E6CFEEFFE82EFAD7EF6A28EC10
:109D40001EF001EE6DF0020E016E5EC52FF05DC5D6
:109D50002EF05CC52DF05BC52CF0030EFEEC00F080
:109D6000EF6A04EEA4F0290EF76E560EF66ED9ECEB
:109D700002F011EE6DF0320EE75204E0E6CFEEFF96
:109D8000E82EFAD7EF6A28EC1EF001EE6DF0020E15
:109D9000016E6EC52FF06DC52EF06CC52DF06BC534
:109DA0002CF0030EFEEC00F0EF6A04EEA4F0290E96
:109DB000F76E660EF66ED9EC02F011EE6DF0320E13
:109DC000E75204E0E6CFEEFFE82EFAD7EF6A28EC80
:109DD0001EF001EE6DF0020E016E4EC52FF04DC566
:109DE0002EF04CC52DF04BC52CF0030EFEEC00F010
:109DF000EF6A04EEA4F0290EF76E760EF66ED9EC3B
:109E000002F011EE6DF0320EE75204E0E6CFEEFF05
:109E1000E82EFAD7EF6A28EC1EF001EE6DF0020E84
:109E2000016E62C52FF061C52EF060C52DF05FC5D3
:109E30002CF0030EFEEC00F0EF6A04EEA4F0290E05
:109E4000F76E860EF66ED9EC02F011EE6DF0320E62
:109E5000E75204E0E6CFEEFFE82EFAD7EF6A28ECEF
:109E60001EF001EE6DF0020E016E72C52FF071C58D
:109E70002EF070C52DF06FC52CF0030EFEEC00F037
:109E8000EF6A04EEA4F0290EF76E960EF66ED9EC8A
:109E900002F011EE6DF0320EE75204E0E6CFEEFF75
:109EA000E82EFAD7EF6A28EC1EF001EE6DF0020EF4
:109EB000016E52C52FF051C52EF050C52DF04FC583
:109EC0002CF0030EFEEC00F0EF6A04EEA4F0290E75
:109ED000F76EA60EF66ED9EC02F011EE6DF0320EB2
:109EE000E75204E0E6CFEEFFE82EFAD7EF6A28EC5F
:109EF0001EF001EE6DF0020E016E66C52FF065C515
:109F00002EF064C52DF063C52CF0030EFEEC00F0BE
:109F1000EF6A04EEA4F0290EF76EB60EF66ED9ECD9
:109F200002F011EE6DF0320EE75204E0E6CFEEFFE4
:109F3000E82EFAD7EF6A28EC1EF001EE6DF0020E63
:109F4000016E76C52FF075C52EF074C52DF073C562
:109F50002CF0030EFEEC00F0EF6A04EEA4F0290EE4
:109F6000F76EC60EF66ED9EC02F011EE6DF0320E01
:109F7000E75204E0E6CFEEFFE82EFAD7EF6A28ECCE
:109F80001EF001EE6DF0020E016E56C52FF055C5A4
:109F90002EF054C52DF053C52CF0030EFEEC00F04E
:109FA000EF6A04EEA4F0290EF76ED60EF66ED9EC29
:109FB00002F011EE6DF0320EE75204E0E6CFEEFF54
:109FC000E82EFAD7EF6A28EC1EF0050125530001B0
:109FD000D8A4F6EF4FF004EEA4F0290EF76EE60ECB
:109FE000F66ED9EC02F0EF6A28EC1EF0010E0501C6
:109FF000255D0001D8A408EF50F004EEA4F0290E6E
:10A00000F76EFC0EF66ED9EC02F0EF6A28EC1EF04B
:08A0100012009CEC48F0120064
:020000040030CA
:03000100861A0F4D
:020005008181F7
:060008000FC00FE00F40E5
:00000001FF
